:100000000C9445010C949A350C94520E0C94620198
:100010000C9462010C9462010C9462010C946201D4
:100020000C9462010C9462010C9462010C94C01057
:100030000C9462010C94292F0C94632F0C948C2F38
:100040000C9462010C9462010C9462010C94673769
:100050000C94620131313056332E333500000001EB
:100060000000060000FF00000F02000C0014010158
:100070000400001450040100000000000000000013
:1000800000000000010003E8000000000000000381
:10009000E800000000000200FA0600070000FF0070
:1000A0000037060002800000000000002107101049
:1000B0000504030206100D0C0B0A2E1005040302A2
:1000C00006100D0C0B0A2E100504030206100D0C71
:1000D0000B0A2E1111111111111111111111111100
:1000E0001111111111111111111111111111110011
:1000F0000404040808080C0C0C1010101414181830
:10010000181C1C1C20202020242424282828282CCB
:100110002C2C2C30303030343434343438383838B7
:10012000383838383C3C3C3C3C3C3C3C3C3C3C1843
:10013000180B0B0C0C0B0C0B040208040C1803031B
:10014000030801010101010804040101000000008D
:1001500000000C10140808090A0B0C08080C090A06
:100160000B0C0D0E080808090A0A0A0A0A0B0C0CE7
:1001700000010405030647401D1B1C1B14133322FA
:1001800019100C080603016744332219100C0803E8
:10019000524F5200000106524F4C000002064D53D0
:1001A00054000003024D5650000004075341500014
:1001B0000005074741500000060353544150000713
:1001C00003525341500008035347500000090747AA
:1001D000475000000A0353544750000B0352534743
:1001E00050000C0352465300000D0353494F0000CA
:1001F0000E0747494F00000F0353414300001D07FE
:1002000053434F00001E0747434F00001F03434363
:100210004F0000200355463000004007554631008E
:10022000004107554632000042075546330000435F
:10023000075546340000440755463500004507552C
:100240004636000046075546370000470752554ED0
:100250000000810553544F5000800042494E000079
:100260008B0000000000000000535441545553001F
:1002700053544F5000535441525400434F4F524433
:100280000052454C00414253000011241FBECFE5EF
:10029000D8E0DEBFCDBF11E0A0E6B0E0ECEFFAE7BA
:1002A00002C005900D92A031B107D9F717E0A0E187
:1002B000B1E001C01D92AF36B107E1F70E946401C1
:1002C0000C947D3D0C940000EF92FF920F931F93CE
:1002D000CF93DF93CDB7DEB724970FB6F894DEBF88
:1002E0000FBECDBF0E94150F82E00E9499100E94A0
:1002F0008F0F8DB18F738DB981E887BB30E020E01F
:1003000018BA00000000000096B380E888BB000027
:1003100000000000B69B02C096FF2F5F3F5F3A309F
:1003200079F72A3039F560E089E090E00E94061004
:1003300060E080E090E00E9406101A82198205C0F9
:1003400089819A8101969A83898389819A818F5FB5
:100350009F4FB1F7C0981A82198205C089819A818E
:1003600001969A83898389819A818F5F9F4FB1F724
:10037000C09AE3CF0E94150F82E00E9499100E945C
:10038000640E0E941B110E948F0FAB980E94560FA3
:100390000E946C0F80E090E00E94FE0F843E09F402
:1003A000DBC0C0980E94483060E089E090E00E9485
:1003B000061040E16DE570E080E090E00E944B1097
:1003C00061E08AE491E00E94061060E08BE491E035
:1003D0000E94061060E08CE491E00E94061060E04C
:1003E0008DE491E00E94061062E08EE491E00E94AC
:1003F000061060E08FE491E00E94061060E080E566
:1004000091E00E94061060E081E591E00E940610F4
:100410000E9423104DE26CE770E08DE390E00E94B3
:100420004B104DE26CE770E08AE690E00E944B10C2
:100430004DE26CE770E087E990E00E944B1043E0EA
:1004400069EA70E084EC90E00E944B1043E06CEAB3
:1004500070E087EC90E00E944B1040E86FEA70E09B
:100460008AEC90E00E944B1064E68AE591E00E94DD
:10047000061060E08BE591E00E94061064E68CE5D2
:1004800091E00E94061060E08DE591E00E94061068
:1004900064E68EE591E00E94061060E08FE591E051
:1004A0000E94061060E080E691E00E94061060E085
:1004B00081E691E00E94061060E082E691E00E94F1
:1004C000061060E083E691E00E94061060E084E69A
:1004D00091E00E94061060E085E691E00E9406101F
:1004E00060E08DEF93E00E94061060E08EEF93E0F5
:1004F0000E94061060E08FEF93E00E94061060E01B
:1005000086E691E00E94061068E087E691E00E948E
:10051000061060E088E691E00E94061068E089E637
:1005200091E00E94061060E08AE691E00E940610C9
:1005300068E08BE691E00E94061081E090E00E9466
:10054000FE0FEEE5F0E0E4918E1729F464EE80E012
:1005500090E00E940610C09A81E090E00E94FE0F99
:100560000E94A12F8AE090E00E94FE0F8093BD04BC
:10057000882311F00E946B388EE70E94350B00E053
:10058000802F80610E94350B802F88610E94350B7F
:10059000802F84600E94350B802F86600E94350B6F
:1005A000802F84610E94350B005E003649F70E945F
:1005B000B4090E947310EE24FF24C70125E0880FC0
:1005C000991F2A95E1F78D600E94D00F082F10E047
:1005D000C80101960E94FE0F8C83C80102960E94FA
:1005E000FE0F8B836B817C818E2D0E947008C7016A
:1005F00085960E94FE0F682F8E2D0E94CD0F0894C5
:10060000E11CF11C83E0E816F104B9F62FEF4FEF7F
:1006100060E086E10E94D3052FEF4FEF60E086E3B4
:100620000E94D3052FEF4FEF60E086E50E94D305CF
:100630008AE491E00E94FE0F80932E078BE491E004
:100640000E94FE0F80932F078CE491E00E94FE0F22
:10065000809330078DE491E00E94FE0F8093310774
:100660008EE491E00E94FE0F8093E6068FE491E015
:100670000E94FE0F8093E70680E591E00E94FE0F46
:100680008093E80681E591E00E94FE0F8093E906E1
:10069000E0902E07F0902F0700913007109131075E
:1006A00085E090E00E94FE0FB801A70190E00E9453
:1006B00093348AE591E00E94FE0F80930F078BE54B
:1006C00091E00E94FE0F809310078CE591E00E945C
:1006D000FE0F809311078DE591E00E94FE0F80933D
:1006E00012078EE591E00E94FE0F809313078FE5BD
:1006F00091E00E94FE0F8093140780E691E00E9433
:10070000FE0F8093F10681E691E00E94FE0F809338
:10071000F20682E691E00E94FE0F8093F30683E6E4
:1007200091E00E94FE0F8093F40684E691E00E941F
:10073000FE0F8093F50685E691E00E94FE0F809300
:10074000F6068DEF93E00E94FE0F809316078EEF62
:1007500093E00E94FE0F809317078FEF93E00E94B3
:10076000FE0F8093180786E691E00E94FE0F8093AB
:10077000570187E691E00E94FE0F8093580188E6BA
:1007800091E00E94FE0F8093590189E691E00E945A
:10079000FE0F80935A018AE691E00E94FE0F80933B
:1007A0005B018BE691E00E94FE0F80935C0182E08A
:1007B00090E00E94FE0F0E94283783E090E00E94A4
:1007C000FE0F80FF03C082E080935E0183E090E033
:1007D0000E94FE0F82958F7080935F010E94A82E69
:1007E0000E94FE0378940E948E060E9421110E94AE
:1007F0006B0B0E943F290E940404F5CF81E0809397
:10080000D1051092B20608958091320781FF07C08A
:100810008091B2068F3F19F08F5F8093B20680916E
:10082000D105813051F48091B2068F3030F0C098FC
:100830001092B20682E08093D1058091D10582307A
:1008400051F48091B206853030F0C09A1092B20611
:1008500081E08093D105089508950895089508953D
:10086000089508950895CF92DF92EF92FF920F932B
:100870001F93CF93DF93CDB7DEB729970FB6F894C8
:10088000DEBF0FBECDBF82E00E9448118CE090E039
:100890000E94FE0F898382E090E00E94FE0F8A830F
:1008A00081E88B8381E48C838091CB068D8380915A
:1008B000CA068E838091CC068F838091CE0688876E
:1008C00019868E010F5F1F4F680189E0E82EF12C19
:1008D000EC0EFD1E8985F8019081890F8987809132
:1008E0005E01882319F480810E94ED2F0F5F1F4F56
:1008F0000E151F0579F780915E01882319F489850B
:100900000E94ED2F80915E01882319F0C6010E949C
:100910005E3929960FB6F894DEBF0FBECDBFDF91CA
:10092000CF911F910F91FF90EF90DF90CF9008959E
:10093000682F70E080FD2FC0CB018076907035E08D
:10094000959587953A95E1F7E82FCB018F799070CF
:100950008431910529F4F0E0E55DF84F2083089596
:100960008630910541F4F0E0EE0FFF1FEC52F94F95
:10097000208341830895089771F4F0E0EE0FFF1F84
:10098000EB5DF84F2083418343FF05C08081918157
:10099000906F918380830895EF92FF920F931F933E
:1009A000182F062FF42EE22E0E9498048BB78F7B0F
:1009B0008BBFC398812F0E94A810802F0E94A8107F
:1009C0008F2D0E94A8108E2D0E94A810C39A8BB75D
:1009D00080648BBF1F910F91FF90EF900895CF928D
:1009E000DF92EF92FF920F931F93CF93DF937C01DF
:1009F0006B01FC01808190E09C012F793070211502
:100A0000310519F028303105E1F4EC01C076D070E1
:100A100045E0D595C7954A95E1F7C33090F48C2F02
:100A20008B5E0E948510682F8C2F0E94CD0FEC2FBB
:100A3000F0E0DF01AA53B94F83E08C93E750F94F00
:100A40001082F70123814281618180810E94980494
:100A50008BB78F7B8BBFC398C0E0D0E086010C0FB3
:100A60001D1FF701EC0FFD1F80810E94A810F801E7
:100A700080832196C430D10589F7C39A8BB78064EF
:100A80008BBF80E090E0DF91CF911F910F91FF909D
:100A9000EF90DF90CF9008955F926F927F928F9248
:100AA0009F92AF92BF92CF92DF92EF92FF920F93FD
:100AB0001F93CF93DF93CDB7DEB728970FB6F89487
:100AC000DEBF0FBECDBF1A829CE0899FC0011124FA
:100AD000B0E85B2E580E00E010E070E0A4E0AA2E13
:100AE000B12CA622B722F2E0CF2ED12CC622D722DB
:100AF000E1E0EE2EF12CE622F72255E0652E712C76
:100B00006C0E7D1E4E010894811C911CA114B10431
:100B100089F0063020F4E114F10421F006C0C1147C
:100B2000D10419F490E180E102C091E181E18B836D
:100B30009C830CC0C80185539F4F0E94FE0F8B837E
:100B4000C80186539F4F0E94FE0F8C83902F002375
:100B500011F0063011F480E18C839A3019F48B8106
:100B600080628B83950D9983B301C4010E94EF04C9
:100B70000E5F1F4F0C30110549F628960FB6F894FA
:100B8000DEBF0FBECDBFDF91CF911F910F91FF90C0
:100B9000EF90DF90CF90BF90AF909F908F907F901D
:100BA0006F905F9008953F924F925F926F927F9205
:100BB0008F929F92AF92BF92CF92DF92EF92FF926D
:100BC0000F931F93CF93DF93CDB7DEB728970FB660
:100BD000F894DEBF0FBECDBFC82E562E442E322E47
:100BE00090E09C012F7930702115310521F02830DB
:100BF000310509F061C08076907045E09595879544
:100C00004A95E1F7D82E82E08D1508F455C0ED2CF9
:100C1000FF24F701EE0FFF1FDF01AF50B94F8D9199
:100C20009C91E25BFE4F91838083F701EC5AFE4F6B
:100C30008081882371F110821A828CE0D89EC001D5
:100C400011248C0100581F4F2CE8A22EB12CA80EA5
:100C5000B91E85E0682E712C6C0E7D1E4E01089425
:100C6000811C911C13C00983C801855B9F4F0E94A2
:100C7000FE0F8B83C801865B9F4F0E94FE0F8C8303
:100C8000B301C4010E94EF040E5F1F4F0A151B053C
:100C900050F38D2D8B5E0E948510682F8D2D0E9444
:100CA000CD0FF701EA53F94F83E08083E9EFF6E0D7
:100CB000EE0EFF1EF7011082232D442D652D8C2D85
:100CC0000E9498048BB78F7B8BBFC3988C2D0E949A
:100CD000A810852D0E94A810842D0E94A810832D95
:100CE0000E94A810C39A8BB780648BBF28960FB65A
:100CF000F894DEBF0FBECDBFDF91CF911F910F9152
:100D0000FF90EF90DF90CF90BF90AF909F908F902B
:100D10007F906F905F904F903F900895AF92BF92F9
:100D2000CF92DF92EF92FF920F931F93CF93DF93B7
:100D3000CDB7DEB72A970FB6F894DEBF0FBECDBF92
:100D40001092BB061092BC061092BD068091C4069C
:100D5000882311F083995FC0809110018F5F809389
:100D60001001833010F0109210018EE090E00E948C
:100D7000FE0F8F5F8093C406809110018295880FCB
:100D8000807E8B608F838E010D5F1F4F67E0C62EC4
:100D9000D12CCC0EDD1EB801C6010E94EF048B8160
:100DA0008093C5068D8183FF02C0806F8D838D8106
:100DB0008A838E818983E0911001F0E0EE0FFF1F9E
:100DC000E254F94F89819A8191838083839923C06A
:100DD000EE24FF2458011E2D1295110F107E812F35
:100DE00087618F83B501C6010E94EF04F701E554C6
:100DF000F94F8E81808316611F838FEF89878A87E1
:100E0000B501C6010E94EF040894E11CF11C83E0C7
:100E1000E816F10401F72A960FB6F894DEBF0FBE6C
:100E2000CDBFDF91CF911F910F91FF90EF90DF9099
:100E3000CF90BF90AF900895CF93DF93EC0182E005
:100E400090E00E94FE0F809324019091210199234C
:100E500059F08091320780FF03C091509093210197
:100E60008091200181600EC080912301882339F098
:100E70008091200180618093200110922301809154
:100E800020018E7F80932001809123018823F1F53A
:100E900081E191E00E94C2338823C1F120911401C5
:100EA00030911501409116015091170180912E0744
:100EB00090912F07A0913007B0913107281739077B
:100EC0004A075B0719F580911101873008F480C04B
:100ED0009E01295F3F4F809124018F83E8E1F1E07B
:100EE000DE0180818D93E90188819191890F88834A
:100EF00081E0EF31F807A9F780911101873011F4F3
:100F000081E001C082E08093DE066DC08091230104
:100F1000882379F468E0CE010E943437882349F0B1
:100F20008F8190912401890F8F8381E08093150731
:100F30005AC00E94C92F8F3F31F4809120018061F7
:100F4000809320013AC085E291E00E94093081300F
:100F5000A1F584E18093210120912301222329F42A
:100F6000809125018093220125C0909122018091DA
:100F700024019817D1F430912001932F946090931D
:100F8000200191FD12C0C20FD11D21978091250132
:100F90008883283051F494FF04C09F7E90932001F1
:100FA00006C036603093200102C0283018F010923D
:100FB000230103C02F5F209323011092DE061092BD
:100FC00015078091200184FF06C08F7E8093200149
:100FD0008FEF9FEF0AC081FD03C080E090E005C065
:100FE0008D7F8093200181E090E0DF91CF91089583
:100FF000FB0120813181280F391F359527953183D9
:101000002083C9010895FF920F931F93F62E8160EC
:101010008093DA060FED16E0B8018AED96E00E94A3
:10102000EF040F0D111DF801808190E01F910F91C9
:10103000FF90089581608093DA066FED76E08AED87
:1010400096E00E94EF048091E20690E008958160AE
:101050008093DA066FED76E08AED96E00E94EF0469
:101060002091E10630E0522F44278091E20690E083
:10107000482B592B23FD02C0CA010895CA01906F65
:101080000895CF93DF93CDB7DEB724970FB6F894CA
:10109000DEBF0FBECDBF81608093DA066FED76E0D4
:1010A0008AED96E00E94EF049091E00697FF03C05E
:1010B0008FEF8C8301C01C829B838091E1068A8321
:1010C0008091E206898369817A818B819C81249653
:1010D0000FB6F894DEBF0FBECDBFDF91CF9108955C
:1010E000CF92DF92FF920F931F93CF93DF93CDB7F1
:1010F000DEB721970FB6F894DEBF0FBECDBF8B01D0
:10110000F82EF294FF0C70EEF7228F2D89618093F8
:10111000DA066FED76E08AED96E00E94EF04C801F2
:101120008070987F892B19F08FEF9FEF57C08091C7
:10113000E106982F9F709C5F82958F70981B0F3FE0
:101140001105F9F0F4F06801191694F0412F5527B4
:10115000202F60E08F2D8C600E94D30520E04FE7A8
:1011600060E08F2D82610E94D30581E090E036C05F
:10117000D594C79491508FEFC816D104E1F0DCF0FC
:10118000E3CF68019D3094F0412F5527202F60E078
:101190008F2D8C600E94D3052DE040E060E08F2D04
:1011A00082610E94D30582E090E018C0CC0CDD1C67
:1011B0009F5FC7FEE7CF412F5527202F60E08F2D7F
:1011C0008C6099830E94D3059981292F4C2D60E072
:1011D0008F2D82610E94D30580E090E021960FB6AA
:1011E000F894DEBF0FBECDBFDF91CF911F910F915D
:1011F000FF90DF90CF9008950F931F93062F182F25
:101200001295110F107E812F85618093DA066FEDA4
:1012100076E08AED96E00E94EF04202F4091E106EF
:1012200060E0812F84610E94D3051F910F91089582
:10123000CF93DF93CDB7DEB724970FB6F894DEBF18
:101240000FBECDBF49835A836B837C8329814A813A
:101250006B810E94D30524960FB6F894DEBF0FBEB3
:10126000CDBFDF91CF9108951F93182F62E00E94A8
:10127000FC081295110F107E40E050E060E070E035
:10128000812F88600E94180940E050E060E070E023
:10129000812F8A600E9418091F9108958295880FF6
:1012A000807E40E050E060E070E088600E941809B5
:1012B0000895E82FF0E0EE0FFF1FE45AF84F408149
:1012C0005181662329F002C0559547956A95E2F74A
:1012D000509541955F4F662757FD6095762F829513
:1012E000880F807E88600E9418090895E82FF0E03A
:1012F000EE0FFF1FE45AF84F40815181662329F019
:1013000002C0559547956A95E2F7662757FD6095A7
:10131000762F8295880F807E88600E941809089534
:101320000F931F93CF93DF93CDB7DEB722970FB6FE
:10133000F894DEBF0FBECDBF8C0101970E94FE0F57
:10134000FE0131968183C8010E94FE0F8983898145
:101350009A8122960FB6F894DEBF0FBECDBFDF9103
:10136000CF911F910F910895CF92DF92EF92FF924C
:101370000F931F93CF93DF93CDB7DEB728970FB6A8
:10138000F894DEBF0FBECDBF1A820BEC10E085E0F3
:10139000C82ED12CCC0EDD1E7E010894E11CF11C60
:1013A000802F8B548983C8010E94FE0F8B83C80154
:1013B00001970E94FE0F8C83B601C7010E94EF04C3
:1013C0000E5F1F4F81E00B34180751F728960FB6B8
:1013D000F894DEBF0FBECDBFDF91CF911F910F916B
:1013E000FF90EF90DF90CF9008951F9390912C0184
:1013F00080912B01981719F480E090E040C0E92F0C
:10140000F0E0EF5BFE4F1081892F8F5F80932C01FE
:101410008A3011F410922C01ECE1F7E0119287E090
:10142000E532F807D9F78CE090E00E94FE0F809338
:101430001C0782E090E00E94FE0F80931D0780E869
:1014400080931E078AE880931F071093230720913B
:101450001A07233019F4EDE1F7E005C080911C076D
:1014600080932407F8CF819190912407890F80936E
:10147000240787E0E432F807B1F7822F90E01F914C
:101480000895EF92FF920F931F938B01E82EFF2494
:10149000C70125E0880F991F2A95E1F788610E940E
:1014A0001A08877002C0000F111F8A95E2F7612F9A
:1014B000772767FD7A95C7014C960E940610602F2A
:1014C000C7014F960E9406101F910F91FF90EF9059
:1014D0000895CF92DF92EF92FF920F931F93CF93D5
:1014E000DF93CDB7DEB728970FB6F894DEBF0FBEF7
:1014F000CDBF1A820BE011E035E0C32ED12CCC0E0B
:10150000DD1E7E010894E11CF11C802F8A54898322
:10151000B601C7010E94EF046F81C8010E94061046
:101520006885C80101970E9406100E5F1F4F81E079
:101530000B34180751F728960FB6F894DEBF0FBE8C
:10154000CDBFDF91CF911F910F91FF90EF90DF9072
:10155000CF900895CF92DF92EF92FF920F931F9357
:10156000CF93DF93CDB7DEB728970FB6F894DEBFE1
:101570000FBECDBF1A820BEC10E045E0C42ED12C7B
:10158000CC0EDD1E7E010894E11CF11C802F8A54D4
:101590008983B601C7010E94EF046F81C8010E94D0
:1015A00006106885C80101970E9406100E5F1F4F44
:1015B00081E00B34180751F728960FB6F894DEBF78
:1015C0000FBECDBFDF91CF911F910F91FF90EF9094
:1015D000DF90CF9008950F931F93CF93DF93082F41
:1015E000816007FD24C08093DA066FED76E08AED16
:1015F00096E00E94EF04802F0E94D00FCFEDD6E03E
:10160000002711270C1B1D0B080F111D6981C80134
:101610008C0F9D1F0E940610823019F482E090E02A
:101620001FC0219686E0C23ED80781F717C080937D
:10163000DA066FED76E08AED96E00E94EF0410E0A6
:101640006091E106C801855B9F4F0E940610609182
:10165000E206C801865B9F4F0E94061080E090E082
:10166000DF91CF911F910F910895FF920F931F93D8
:10167000CF93DF93CDB7DEB728970FB6F894DEBFD0
:101680000FBECDBFF82E0E94D00F082F10E0F982B8
:10169000C8010E94FE0F8A83C80101960E94FE0FB6
:1016A0008B83C80102960E94FE0F8C83BE016B5F84
:1016B0007F4FCE0101960E94EF0480E090E02896D3
:1016C0000FB6F894DEBF0FBECDBFDF91CF911F9153
:1016D0000F91FF9008952F923F924F925F926F92D9
:1016E0007F928F929F92AF92BF92CF92DF92EF92B2
:1016F000FF920F931F93CF93DF93CDB7DEB724975D
:101700000FB6F894DEBF0FBECDBF86E090E00E941A
:10171000FE0F8A8380913D018F5F80933D01815050
:10172000823010F010923D0180912601882369F4E7
:1017300080E68093DA066FED76E08AED96E00E940F
:10174000EF041092270181E01BC08130E1F481E6B3
:101750008093DA066FED76E08AED96E00E94EF0462
:101760008091DF0686FD72C08091E10686958095A6
:1017700087708093E3068091E2068093FC0682E006
:101780008093260163C0823009F060C080912701F8
:10179000A82FB0E0FD01EA5EF84F9081992309F48B
:1017A00050C0FD01ED51F94F8081891708F449C0FF
:1017B00015E0AA0FBB1F1A95E1F78A2F8A600E94D5
:1017C0002708BC01892B09F43FC0A09127014A2FAB
:1017D00050E0FA01E55DF84F8081FA01EE0FFF1F3E
:1017E000882319F0EB5DF84F02C0EC52F94F2081CD
:1017F0003181CB0177FF03C0909581959F4F37FFD3
:1018000003C0309521953F4F82179307E9F4FA0101
:10181000E25CFE4F8081823078F08A2F0E9434098A
:10182000E0912701F0E0DF01A750B94F81E08C93F0
:10183000E25CFE4F108208C08F5F80831092260109
:1018400003C0A25CBE4F1C92109226018091320709
:1018500080FFAFC180E00E947D3181E00E947D3138
:1018600082E00E947D318DE78093DA066FED76E0AD
:101870008AED96E00E94EF0410912C01E0912B017B
:1018800070915D01A0E0B0E041E050E00A2E02C09E
:10189000440F551F0A94E2F7642F842F8723D9F051
:1018A0008091DF0690E09D01220F331F02C09595C5
:1018B00087952A95E2F780FF0EC08E2F8F5F8A30C2
:1018C00009F480E0811729F0F0E0EF5BFE4F4083E0
:1018D000E82F609576231196A330B105A9F6E09321
:1018E0002B0170935D018091320781FFAEC00BE444
:1018F00011E0E4E56E2EE1E07E2E78E2872E71E0C5
:10190000972E6FE0462E67E0562E56ECA52E56E039
:10191000B52E1C821B8240E8C42E36E8332EDB80B5
:101920008B819C8125E0880F991F2A95E1F78A60B9
:101930000E9427087C018091320782FF1EC0F501BA
:101940008081E114F10461F0833041F08D2D8B5ED4
:101950000E948510682F8B810E94CD0F83E00BC001
:10196000882341F48B810E948510682F8B810E940F
:10197000CD0F03C08150F5018083F20120813181B8
:10198000FFEF2F3F3F07A9F4F8018081823009F46F
:1019900041C021E145E060E08C2D0E94CC0421E1B2
:1019A0004DE060E0832D0E94CC0482E0F80180834A
:1019B00031C0C701F7FE03C0909581959F4FF80194
:1019C00040818217930794F0413021F127E045E0F0
:1019D00060E08C2D0E94CC042FE04DE060E0832D70
:1019E0000E94CC0481E0F801808310C0442391F070
:1019F00020E145E060E08C2D0E94CC0420E14DE028
:101A000060E0832D0E94CC04F8011082F301108263
:101A1000F40110828B819C8101969C838B839CE0D6
:101A2000C90E390E0F5F1F4F0894611C711C08947A
:101A3000811C911CE2E0F0E04E0E5F1E0894A11C98
:101A4000B11CF4EACF1609F06ACF81EF282E86E0A8
:101A5000382E08E2C02E01E0D02E17E5412E11E00D
:101A6000512EB4E56B2EB1E07B2EAEE48A2EA1E0C0
:101A70009A2EAA24BB248AE88983C501F5E0880F41
:101A8000991FFA95E1F78A600E9427087C0197FF69
:101A900004C0F094E194F108F394F1018081918104
:101AA000892B39F1E114F10421F5F4018081918150
:101AB0000097D9F4F30180818823D9F419811A5051
:101AC00000E020E140E160E0812F0E94CC040E5F45
:101AD0001E5F0C30B1F720E140E360E089810E9495
:101AE000CC0481E0F301808304C00197F401918369
:101AF0008083AA2009F044C0F2018081918100977F
:101B000009F4AFC0E816F90608F4ABC0F60180810D
:101B1000882309F0A6C081E0808300EC10E02CE26D
:101B20004CE260E0802F0E94CC040E5F1F4FF1E07A
:101B300000301F0709F495C0F2CF892B09F5F60193
:101B400080818823E9F01082EAE0EE2EE1E0FE2EAB
:101B5000C7010E94FE0F182FC70101960E94FE0FB9
:101B6000212F482F60E08E2D8A540E94CC0482E001
:101B700090E0E80EF91E9AE4E91691E0F90641F7C3
:101B80000894A11CB11CE2E0F0E02E0E3F1E089468
:101B9000C11CD11C4E0E5F1EF981F45FF9830894BD
:101BA000611C711C82E090E0880E991EFE3A09F0DB
:101BB00064CF8091C9068823F9F484E08093C90634
:101BC00068E08FEF96E00E94700FA7B1B0E0AA0F17
:101BD000BB1FA35DBE4FE7B1F0E0EE0FFF1FE1506A
:101BE000F94F8D919C91119720813181820F931F24
:101BF000959587958D939C9390913D01E92FF0E009
:101C0000E251F94F8081882319F0892F0E948B318E
:101C10009A81992311F1EA81E13019F49A9906C069
:101C20001CC0FA81F230C9F49A9917C0AB9A81E0CE
:101C30008093190700E010E062E0802F0E94FC080A
:101C4000802F0E944E09F801E251F94F10820F5F78
:101C50001F4F0330110569F0EFCFAB9810921907B1
:101C600008C0F20180819181E816F90608F467CF77
:101C700064CF24960FB6F894DEBF0FBECDBFDF91C0
:101C8000CF911F910F91FF90EF90DF90CF90BF9079
:101C9000AF909F908F907F906F905F904F903F900C
:101CA0002F9008951F920F920FB60F9211248F93C9
:101CB00081E08093CD068F910F900FBE0F901F9003
:101CC00018951092CD0608951F93CF93DF93CDB74B
:101CD000DEB722970FB6F894DEBF0FBECDBF23E06C
:101CE00040E060E084E10E94CC0423E040E060E05A
:101CF00084E30E94CC0423E040E060E084E50E949D
:101D0000CC0420E040E060E08AE00E94CC0420E0C7
:101D100040E060E08AE20E94CC0420E040E060E025
:101D20008AE40E94CC0410E002C01431A1F020E04B
:101D300040E060E0812F0E94CC0420E040E060E0C1
:101D4000812F80620E94CC0420E040E060E0812F7F
:101D500080640E94CC041E5F1C3138F320E040E018
:101D600060E08EE70E94CC0410E020E040E060E0FC
:101D7000812F80680E94CC041E5F1038B1F72FEFCE
:101D800047E060E08AE00E94CC041A82198206C013
:101D9000000089819A8101969A83898389819A8139
:101DA000885B9B40ACF320E040E060E08AE00E946A
:101DB000CC048BB78F7B8BBFC39883E00E94A810A5
:101DC00080E00E94A8108093D10680E00E94A810B5
:101DD0008093D00680E00E94A8108093CF06C39A1B
:101DE0008BB780648BBF20E040E060E082E00E941F
:101DF000CC048091CF069091D006A091D106B091ED
:101E0000D206805D9740A040B04010F480E101C050
:101E100088E08093D30622960FB6F894DEBF0FBEFB
:101E2000CDBFDF91CF911F910895CF93DF93CDB7B1
:101E3000DEB722970FB6F894DEBF0FBECDBF8EEF90
:101E40008ABB8CE08BBB8DEB87BB8FE188BB8CEFB3
:101E500084BB83EF85BB82EF81BB85E082BBDB98CF
:101E60001A82198206C0000089819A8101969A839C
:101E7000898389819A8184369105ACF3DB9A1A8231
:101E8000198206C0000089819A8101969A8389830C
:101E900089819A8184369105ACF322960FB6F89425
:101EA000DEBF0FBECDBFDF91CF91089581B3806BB0
:101EB00081BB81EF8FBD81E08EBD81E785BD089537
:101EC000882319F41BBC6ABD0895813019F419BC2C
:101ED00068BD089563BD089517B886EC86B9089566
:101EE00044B150E025B1E7B1F0E0EE0FFF1FE80F7D
:101EF000F91F30E0322F2227242B352B318320830A
:101F000087B190E070E0615070408617970724F425
:101F100087B18F5F87B901C017B8369A08950895C1
:101F2000882309F4D99A0895882309F4D998089543
:101F3000882319F080E090E0089589B390E08170E3
:101F400090700895482F662359F02BB381E090E0FC
:101F500002C0880F991F4A95E2F7282B2BBB0895E2
:101F60002BB381E090E002C0880F991F4A95E2F7F9
:101F7000809582238BBB0895882319F080E090E040
:101F800008958BB390E09695879581709070089531
:101F90008BBB089580E090E008950E94600F089543
:101FA000282F87FD23C0482F46954F7083E0489F18
:101FB000C001112430E0207630702115310511F474
:101FC000CD961AC02032310519F486599F4F14C09E
:101FD0002034310519F489569F4F0EC04F3019F443
:101FE00087EC90E009C04E3039F404C0265B822FA4
:101FF00090E0089583E090E090E00895DC01E1999D
:10200000FECF0E942F3D802D90E008951F93CF9327
:10201000DF93EC01162F89E090E00E94FE0F8823E9
:1020200031F0C930D10519F082E090E008C0E199A3
:10203000FECFDE01012E0E94373D80E090E0DF916F
:10204000CF911F910895EF92FF921F93CF93DF934B
:102050008DE6E82E80E0F82EC0E1D0E0F701149183
:10206000612FCE010E940610612FCE0101960E94C1
:102070000610612FCE0102960E9406100894E11C02
:10208000F11C2396CD33D10549F7DF91CF911F91F4
:10209000FF90EF900895CF92DF92EF92FF920F930F
:1020A0001F93CF93DF936C017B01042F10E0C0E0FE
:1020B000D0E00CC0FE01EE0DFF1DE4916E2FCE01AD
:1020C0008C0D9D1D0E9406101F5F2196101791F721
:1020D00080E090E0DF91CF911F910F91FF90EF9002
:1020E000DF90CF900895CF93DF93C0E1D0E0CE0191
:1020F0000E94FE0FFE01E05BFE4F80832196CD33F0
:10210000D105A9F7DF91CF910895E0E6F1E0E80F5E
:10211000F11D808190E008958D3218F081E090E00B
:102120000895E82FF0E0E05AFE4F608380E090E0F1
:10213000089583708DB98DB18C658DB9709A1092A8
:102140008D01089580918D0110928D0190E0089588
:102150008FB980E009C0893C31F480918D018160A4
:1021600080938D0103C08F5F779BF5CF769B05C071
:1021700080918D01826080938D018FB190E00895F0
:102180001F920F920FB60F9211248F939F93AF93CC
:10219000BF938091D306883011F482E701C083E2B7
:1021A00082BF80913307882319F0815080933307D1
:1021B0008091C406882319F081508093C4068091D1
:1021C0009101882321F08150809391012BC088E0F8
:1021D0008093910180918E01882319F08150809322
:1021E0008E018091C906882319F081508093C90619
:1021F0008091EA069091EB06A091EC06B091ED0675
:102200000196A11DB11D8093EA069093EB06A09361
:10221000EC06B093ED068091F706882319F0815003
:102220008093F706BF91AF919F918F910F900FBE52
:102230000F901F90189582E083BF81E089BF88BF0F
:1022400008951092320780918E01882301F59AE05B
:1022500090938E0181E08093320780918F018823D3
:1022600021F0815080938F01089590938F0183E036
:102270008093320780919001882321F081508093D0
:10228000900108959093900187E08093320708951C
:102290008093C001089599E0699FA001112490E006
:1022A000837090709C01220F331F280F391F420F3B
:1022B000531F455E5D4F82E0403D580714F04BE1EF
:1022C00052E0CA0108950F931F93CF93DF93CDB7C8
:1022D000DEB728970FB6F894DEBF0FBECDBFE82F4C
:1022E0000D831E832F83388780936E076093380792
:1022F0004093390781E080935A0738853093CB06A5
:102300002F812093CA069E819093CC068D81809365
:10231000CE069093B8018093B7013093BC0120930F
:10232000BB019093BA018093B901F0E0EE0FFF1F5B
:10233000E05AFF4F0190F081E02D8091EC01811176
:1023400009958091CB0687FF03C08FEF8C8301C076
:102350001C828091CA068B838091CC068A838091EF
:10236000CE06898369817A818B819C8128960FB6FC
:10237000F894DEBF0FBECDBFDF91CF911F910F91BB
:1023800008950000089500000895000008950000D9
:102390000895809138078823A9F48091410790918E
:1023A0004207A0914307B09144072091B9013091B1
:1023B000BA014091BB015091BC01820F931FA41F31
:1023C000B51FC4C08130A9F48091410790914207A4
:1023D000A0914307B09144072091B9013091BA010F
:1023E0004091BB015091BC01821B930BA40BB50B18
:1023F000ADC0823099F4609141077091420780919D
:102400004307909144072091B9013091BA0140915E
:10241000BB015091BC010E94A43C31C08330D9F46F
:102420006091410770914207809143079091440762
:102430002091B9013091BA014091BB015091BC018A
:102440000E94EA3C209341073093420740934307A0
:102450005093440783C08430D9F460914107709150
:10246000420780914307909144072091B901309130
:10247000BA014091BB015091BC010E94EA3C6093BB
:10248000410770934207809343079093440766C0C7
:102490008530A9F48091410790914207A0914307AC
:1024A000B09144072091B9013091BA014091BB012C
:1024B0005091BC0182239323A423B52347C08630C7
:1024C000A9F48091410790914207A0914307B091F0
:1024D00044072091B9013091BA014091BB0150915C
:1024E000BC01822B932BA42BB52B30C08730A9F4D1
:1024F0008091410790914207A0914307B091440712
:102500002091B9013091BA014091BB015091BC01B9
:1025100082279327A427B52719C0883069F48091B2
:10252000410790914207A0914307B09144078095DD
:102530009095A095B0950AC0893081F48091B90139
:102540009091BA01A091BB01B091BC018093410769
:1025500090934207A0934307B093440780914107AB
:1025600090914207A0914307B09144072091C20186
:102570003091C3010097A105B10511F4286001C095
:10258000277F3093C3012093C201089580913807BB
:102590008823A9F48091410790914207A0914307B5
:1025A000B091440720916A0730916B0740916C0706
:1025B00050916D07820F931FA41FB51F16C0813065
:1025C000E9F48091410790914207A0914307B091AF
:1025D000440720916A0730916B0740916C07509136
:1025E0006D07821B930BA40BB50B8093410790934F
:1025F0004207A0934307B0934407D8C0823099F4B0
:102600006091410770914207809143079091440780
:1026100020916A0730916B0740916C0750916D07CC
:102620000E94A43C31C08330D9F46091410770917D
:102630004207809143079091440720916A073091A7
:102640006B0740916C0750916D070E94EA3C209304
:102650004107309342074093430750934407A6C075
:102660008430D9F46091410770914207809143070B
:102670009091440720916A0730916B0740916C0755
:1026800050916D070E94EA3C6093410770934207A6
:10269000809343079093440789C08530A9F48091C3
:1026A000410790914207A0914307B09144072091C0
:1026B0006A0730916B0740916C0750916D07822338
:1026C0009323A423B52391CF8630A9F480914107A9
:1026D00090914207A0914307B091440720916A0767
:1026E00030916B0740916C0750916D07822B932BB3
:1026F000A42BB52B7ACF8730A9F480914107909114
:102700004207A0914307B091440720916A07309196
:102710006B0740916C0750916D0782279327A42780
:10272000B52763CF883069F480916A0790916B0771
:10273000A0916C07B0916D0780959095A095B0958C
:102740000AC0893089F48091410790914207A09195
:102750004307B091440780936A0790936B07A09357
:102760006C07B0936D0722C08A3001F520914107B4
:1027700030914207409143075091440780916A0786
:1027800090916B07A0916C07B0916D078093410702
:1027900090934207A0934307B093440720936A079E
:1027A00030936B0740936C0750936D0780914107FE
:1027B00090914207A0914307B09144072091C20134
:1027C0003091C3010097A105B10511F4286001C043
:1027D000277F3093C3012093C2010895EF92FF92A7
:1027E0000F931F93E0904107F09042070091430739
:1027F000109144072091B9013091BA014091BB0179
:102800005091BC012E153F05400751073CF48091C3
:10281000C2019091C30184608C7F0EC08091C2017F
:102820009091C301E216F3060407150719F4897F96
:10283000816002C0887F82609093C3018093C2014F
:102840008091C2019091C301E114F10401051105C9
:1028500011F4886001C0877F9093C3018093C20107
:102860001F910F91FF90EF90089580913807882372
:1028700039F48091C2019091C30183FF7AC060C096
:10288000813039F48091C2019091C30183FD71C000
:1028900057C0823029F48091C2019091C3012CC0AD
:1028A000833039F48091C2019091C30180FD61C0F1
:1028B00047C0843039F48091C2019091C30182FFF6
:1028C00058C03EC0853039F48091C2019091C30157
:1028D00082FD36C011C0863039F48091C2019091DA
:1028E000C30181FF46C02CC0873049F48091C201EA
:1028F0009091C30181FD24C080FF3BC021C088307E
:1029000039F48091C2019091C30184FF32C018C094
:10291000893039F48091C2019091C30185FF29C0AB
:102920000FC08A3039F48091C2019091C30186FFB3
:1029300020C006C08B3069F48091C20187FF19C0A6
:102940008091B7019091B801909336078093350735
:1029500008958C3071F48091C2019091C30190FF71
:1029600008C08091B7019091B80190933607809389
:10297000350708958091B7019091B801909336077B
:102980008093350708952091A3012830B8F4E22FF1
:10299000F0E0EE0FFF1FED56FE4F8091350790914E
:1029A0003607918380832F5F2093A3018091B70125
:1029B0009091B80190933607809335070895E09180
:1029C000A301EE2371F0E150E093A301F0E0EE0FDC
:1029D000FF1FED56FE4F80819181909336078093C3
:1029E0003507089580913807813011F48093920162
:1029F000089580913807813011F410929201089562
:102A000010924007089580913807882339F4809107
:102A1000C2019091C3018F7090701FC0813031F45A
:102A20008091C2019091C3018F7E17C0823031F432
:102A30008091C2019091C3018F7D0FC0833031F42A
:102A40008091C2019091C3018F7B07C0843051F403
:102A50008091C2019091C3018F779093C3018093BD
:102A6000C2010895853049F48091C2019091C3015B
:102A70009E7F9093C3018093C2010895809138078F
:102A8000813041F48091CC068093DF018091CE06A5
:102A90008093E001089508950000089500000895CE
:102AA00000000895000008950000089500000895B2
:102AB00000000895000008950000089500000895A2
:102AC0000000089500000895000008950000089592
:102AD0000000089500000895000008950000089582
:102AE0000000089500000895000008950000089572
:102AF0000000089500000895000008951092400716
:102B0000089580913807813041F48091B701909108
:102B1000B801909336078093350781E08093400792
:102B2000089582E080934007089583E080934007F2
:102B300010923607109235078FEF9FEF9093C701E1
:102B40008093C6011092A301109245071092A40130
:102B500081E08093BF011092C5011092C4011092D0
:102B600041071092420710924307109244071092B7
:102B70009201089510924D071092C5011092C40160
:102B80000895809138078130D9F0813030F082305B
:102B900031F1833009F044C033C080914007809305
:102BA000CB06809145078093CA062091C4013091DD
:102BB000C501832F99278093CC062093CE060895D4
:102BC000809140078093CB06809145078093CA0689
:102BD000809136078093CC06809135070EC0809196
:102BE00044078093CB06809143078093CA06809167
:102BF00042078093CC06809141078093CE060895CA
:102C000080916D078093CB0680916C078093CA06F4
:102C100080916B078093CC0680916A078093CE06E3
:102C200008958091CE0680935D0181E080931A071C
:102C30008091DE06882319F082E080931A07809144
:102C40001507882319F083E080931A07089580916F
:102C50005E01882321F481E080935E010895823033
:102C600019F483E080935E010895809138078130E4
:102C700049F08130A0F0823009F44FC0833009F070
:102C800063C058C04091DD015091DE016091B701F1
:102C90007091B801E9ECF1E020E030E03AC0209119
:102CA000DD013091DE012A30310590F4F901EE0F9B
:102CB000FF1FE753FE4F8091B7019091B8019183B8
:102CC00080832F5F3F4F3093DE012093DD01089515
:102CD00089E0809334070895819191918617970731
:102CE000B1F4F901EE0FFF1FE753FE4F4150504082
:102CF00006C02F5F3F4F8281938181939193241768
:102D00003507B8F35093DE014093DD0108952F5F3E
:102D10003F4F2417350701F708951092DE011092F6
:102D2000DD01E9ECF1E01192119281E0ED3DF8074F
:102D300071F0F9CF1092CB061092CA061092CC0611
:102D40008AE08093CE06089583E080933407089547
:102D500080916307813881F580916407823961F53C
:102D600080916507833A41F580916607843B21F5A0
:102D700080916707853C01F580916807863DE1F405
:102D8000F894C098AB9A89E0E3E0F0E080935700B4
:102D90008491867019F40C9400380895823019F4E7
:102DA0000C94003C0895843019F40C94003E08956E
:102DB000863011F40C94003F0895CF93DF93CDB784
:102DC000DEB728970FB6F894DEBF0FBECDBF809157
:102DD00038078130F1F4809139078A32C1F480914B
:102DE000CE0689838091CC068A838091CA068B8324
:102DF0008091CB068C831D821E821F821886BE01A5
:102E00006F5F7F4F8FEF97E00E94FA302FC084E012
:102E10002BC0882341F5BE016F5F7F4F8FEF97E096
:102E20000E94C4309091CE068981981799F49091B0
:102E3000CC068A81981771F49091CA068B819817F5
:102E400049F49091CB068C81981721F481E080930E
:102E5000CE0602C01092CE061092CB061092CA0681
:102E60001092CC0603C083E08093340728960FB6F7
:102E7000F894DEBF0FBECDBFDF91CF910895809152
:102E80004007882389F1833079F1853069F165EA5B
:102E900071E080913507909136070E94C4302091EF
:102EA0003507309136078091C6019091C70182178E
:102EB000930721F081E08093BF0102C01092BF010F
:102EC0003093C7012093C6012F5F3F4F30933607E1
:102ED0002093350780914007823019F485E0809374
:102EE000400781E090E0089580E090E008958CE054
:102EF00090E00E94FE0F8093AE01809138078823F6
:102F000099F482E08093C00124E530E0AEEAB1E0BC
:102F1000F9018491FD0181832F5F3F4F1196F1E00C
:102F2000A63BBF0761F0F4CF1092CB0681E08093FF
:102F3000CA0683E08093CC0683E28093CE06089590
:102F40002091B7013091B8013093C5012093C4019D
:102F500082E08093C0012F5F374078F487E090E0F3
:102F60000E94FE0F80FD09C06FEA71E08091C401EC
:102F70009091C5010E94C43007C0EEEAF1E01192C1
:102F800081E0E73BF807D9F78CE090E00E94FE0F64
:102F90008093AE01089583E08093400787E090E03E
:102FA0000E94FE0F81FD04C081E080934D0703C0A5
:102FB00088E0809334078091B7019091B801909395
:102FC000C5018093C40108950F931F93CF93DF939E
:102FD000CDB7DEB724970FB6F894DEBF0FBECDBFD6
:102FE000E82FF0E06623C1F189E0689F8001112499
:102FF0009F0123703070C901880F991F820F931FA2
:10300000080F191F055E1D4F82E00F3C180744F0A2
:1030100081E08093340760E070E080E090E026C0BB
:10302000C80102960E94FE0F8B83C80101960E9480
:10303000FE0FFE0131968183C8010E94FE0F898335
:103040008B8187FF03C08FEF8C8301C01C82698155
:103050007A818B819C810AC0EE0FFF1FEE0FFF1F4C
:10306000E25BF84F608171818281938124960FB673
:10307000F894DEBF0FBECDBFDF91CF911F910F91AE
:103080000895CF93DF93CDB7DEB724970FB6F894AA
:10309000DEBF0FBECDBF60913807809139070E9417
:1030A000E41769837A838B839C834C814093CB069E
:1030B0003B813093CA062A812093CC069981909354
:1030C000CE0680915A078823F9F040934407309345
:1030D00043072093420790934107809141079091C5
:1030E0004207A0914307B09144072091C20130915B
:1030F000C3010097A105B10511F4286001C0277F25
:103100003093C3012093C20124960FB6F894DEBF1A
:103110000FBECDBFDF91CF9108958091B7019091FF
:10312000B801825D944041F460E080E090E00E944C
:103130000610F8940C94000008950F931F93CF93FA
:10314000DF93CDB7DEB724970FB6F894DEBF0FBE7E
:10315000CDBF90913807992341F189E0989F800174
:1031600011248091390723E0829FC0011124080FA8
:10317000191F055E1D4F82E00F3C180724F081E007
:103180008093340732C06091CA06C80102960E943B
:1031900006106091CC06C80101960E94061060914D
:1031A000CE06C8010E94061020C08091CA068B83FB
:1031B0009091CC069A839091CE06998387FF03C0A5
:1031C0008FEF8C8301C01C82E0913907F0E0EE0F95
:1031D000FF1FEE0FFF1FE25BF84F89819A81AB81E1
:1031E000BC8180839183A283B38324960FB6F89425
:1031F000DEBF0FBECDBFDF91CF911F910F9108951C
:103200009091380797FF13C0809144078093CB06B5
:10321000809143078093CA06809142078093CC0631
:10322000809141078093CE069F77909338079091C5
:103230003807992329F0923019F0933009F046C0ED
:10324000C39A8BB780648BBFC49A8BB780648BBFE3
:10325000992329F48BB78F7B8BBFAF980DC0923029
:1032600029F48BB78F7B8BBFAE9806C0933021F4C7
:103270008BB78F7B8BBFAD9880913907843030F04E
:103280008091CB060E94A8108093CB0680913907CD
:10329000833030F08091CA060E94A8108093CA063D
:1032A00080913907823030F08091CC060E94A810BE
:1032B0008093CC068091CE060E94A8108093CE0603
:1032C00085B3806E85BB8BB780648BBF80913807D8
:1032D000813051F585B3806E85BB8BB780648BBF21
:1032E000C49A8BB780648BBF8BB78F7B8BBFC3981F
:1032F0008091CB060E94A8108093CB068091CA06CD
:103300000E94A8108093CA068091CC060E94A81043
:103310008093CC068091CE060E94A8108093CE06A2
:10332000C39A8BB780648BBF80915A07882359F169
:103330008091CB06809344078091CA06809343070F
:103340008091CC06809342078091CE0680934107FE
:103350008091410790914207A0914307B0914407A3
:103360002091C2013091C3010097A105B10531F44C
:1033700028603093C3012093C2010895277F3093C2
:10338000C3012093C20108951F9381E080934507F4
:1033900040913807442339F08091B7019091B801EA
:1033A0001816190604F52091BF01222341F08091DF
:1033B000B7019091B8019093BE018093BD01442361
:1033C00091F48091B7019091B8018F5F9F4F51F5B3
:1033D000222341F180914107909142079093BE01D1
:1033E0008093BD011FC08091B7019091B80118165C
:1033F00019061CF020E030E00AC020E08091BD01F9
:103400009091BE01892B09F021E081E02827122F3D
:103410008091C2019091C301222311F0806121C0EB
:103420008F7E1FC08091BD019091BE01892B11F448
:103430001092450780914507882341F08091C6018D
:103440009091C70190933607809335078091C20110
:103450009091C3018F7E9093C3018093C20110E0CD
:1034600025C09093C3018093C2014130F9F460E01C
:103470008DE70E94030890E020913907220F02C0D7
:10348000959587952A95E2F780FF02C0109245072F
:1034900080914507882351F0112341F48091C601A2
:1034A0009091C70190933607809335078091380734
:1034B000823019F563E08DE70E94030890E04091A7
:1034C0003907440F22E030E002C0220F331F4A9533
:1034D000E2F782239323892B11F010924507809104
:1034E0004507882351F0112341F48091C601909142
:1034F000C701909336078093350780913807833052
:10350000F9F463E08DE70E94030890E02091390709
:10351000220F02C0959587952A95E2F780FF02C099
:103520001092450780914507882351F0112341F4FB
:103530008091C6019091C70190933607809335071B
:1035400080913807843009F049C0E0913907E330B1
:1035500050F410924507F0E0E251F94F8081882342
:1035600079F181E028C0E43049F48091EE068823A7
:1035700001F520E030E08091EF0615C0E53059F00C
:10358000E63019F48091EE0608C0E730B9F4809176
:10359000EE06882371F48091EF06882351F420E031
:1035A00030E08091F006882311F021E030E0C9017D
:1035B00002C081E090E08093450702C01092450769
:1035C00080914507882351F0112341F48091C60171
:1035D0009091C70190933607809335071F91089506
:1035E00080913807882341F4E0913907F0E0E251F7
:1035F000F94F81E080830895813081F4809139070B
:10360000E82FF0E0E251F94F9FE0908362E00E94E2
:10361000FC08809139070E944E090895823049F5CF
:10362000E0913907F0E0E251F94FE081E093CE06F6
:1036300080915A078823E9F08E2F90E0A0E0B0E057
:103640008093410790934207A0934307B0934407A8
:103650008091C2019091C301EE2331F48860909370
:10366000C3018093C2010895877F9093C301809323
:10367000C201089562E0809139070E94FC088091A0
:1036800039070E944E090895EF92FF920F931F93FE
:10369000CF93DF9380913907882341F480913807D5
:1036A000873109F001C10E94B409FEC0813009F0E0
:1036B000B0C080913807863038F4C82FD0E0C759A1
:1036C000DE4F8330E1F415C0893038F4C82FD0E0E4
:1036D000CC0FDD1FCC59DE4F12C08C3008F0E1C09A
:1036E000C82FD0E0CC0FDD1FCC0FDD1FCC5ADE4F32
:1036F00006C0CE010E94FE0F8093CD050FC084301E
:1037000031F4CE010E94FE0F8093CC0507C08530B6
:1037100029F4CE010E94FE0F8093CE0580913807D8
:10372000863061F4CE0101960E94FE0F8093D00591
:10373000CE010E94FE0F8093CF05B6C0873061F4A2
:10374000CE0101960E94FE0F8093C905CE010E9412
:10375000FE0F8093C805A8C0883061F4CE010196A1
:103760000E94FE0F8093CB05CE010E94FE0F809336
:10377000CA059AC08930C1F4CE0103960E94FE0F9B
:103780008093B606CE0102960E94FE0F8093B50686
:10379000CE0101960E94FE0F8093B406CE010E94D6
:1037A000FE0F8093B30680C08A30C1F4CE01039629
:1037B0000E94FE0F8093BA06CE0102960E94FE0F71
:1037C0008093B906CE0101960E94FE0F8093B80641
:1037D000CE010E94FE0F8093B70666C08B3009F0C1
:1037E00063C0CE0103960E94FE0F8093C705CE01F1
:1037F00002960E94FE0F8093C605CE0101960E949C
:10380000FE0F8093C505CE010E94FE0F8093C40574
:103810004BC0823009F048C000913807083308F0E7
:1038200043C010E0000F111F000F111FBBE1EB2E72
:10383000B3E0FB2EE00EF11EC7010E94FE0F0E52F8
:103840001A4FF801808380913807C82FD0E0CC0F41
:10385000DD1FCC0FDD1FCD52DA4FC70101960E944C
:10386000FE0F888380913807C82FD0E0CC0FDD1F72
:10387000CC0FDD1FCC52DA4FC70102960E94FE0F1B
:10388000888380913807C82FD0E0CC0FDD1FCC0F84
:10389000DD1FCB52DA4FC70103960E94FE0F8883CB
:1038A00003C0CFEFD3E02BCFDF91CF911F910F91CA
:1038B000FF90EF9008950F931F93CF93DF93809124
:1038C0003907882321F480913807893449F089E049
:1038D00090E00E94FE0F882319F085E08093340762
:1038E00080913907882311F580913807803428F5B5
:1038F000873088F4863011F48EE70AC0880F880F6D
:103900008C590E94EB0A80913807880F880F8A59DA
:103910000E94EB0AF0C0873019F40E94AA0AEBC09B
:10392000873109F0E8C00E94690AE5C0813009F0DA
:103930009FC080913807833020F483E08093340760
:10394000DAC0863038F4C82FD0E0C759DE4F833054
:10395000C9F415C0893038F4C82FD0E0CC0FDD1F72
:10396000CC59DE4F0FC08C3008F0C2C0C82FD0E059
:10397000CC0FDD1FCC0FDD1FCC5ADE4F03C0609192
:10398000CD0509C0843019F46091CC0504C08530A0
:1039900029F46091CE05CE010E940610809138076F
:1039A000863049F46091D005CE0101960E94061040
:1039B0006091CF055BC0873049F46091C905CE01A5
:1039C00001960E9406106091C80550C0883049F4E5
:1039D0006091CB05CE0101960E9406106091CA0548
:1039E00045C08930A9F46091B606CE0103960E94C5
:1039F00006106091B506CE0102960E9406106091F5
:103A0000B406CE0101960E9406106091B3062EC046
:103A10008A30A9F46091BA06CE0103960E9406107E
:103A20006091B906CE0102960E9406106091B80618
:103A3000CE0101960E9406106091B70617C08B3028
:103A400009F059C06091C705CE0103960E94061087
:103A50006091C605CE0102960E9406106091C505D0
:103A6000CE0101960E9406106091C405CE013DC0B2
:103A7000823009F040C0E0913807E833E0F5F0E02B
:103A8000EE0FFF1FEE0FFF1F8F01055E1C4FEE5262
:103A9000FA4F6381C80103960E940610E09138072F
:103AA000F0E0EE0FFF1FEE0FFF1FEE52FA4F6281A4
:103AB000C80102960E940610E0913807F0E0EE0F70
:103AC000FF1FEE0FFF1FEE52FA4F6181C8010196F2
:103AD0000E940610E0913807F0E0EE0FFF1FEE0F96
:103AE000FF1FEE52FA4F6081C8010E94061003C00A
:103AF000CFEFD3E047CFDF91CF911F910F91089582
:103B00000F931F93CF93DF93CDB7DEB728970FB6F0
:103B1000F894DEBF0FBECDBF80913907882309F02E
:103B2000DCC08091380787FD7DC0803408F041C03B
:103B30008630A9F48FE78093DA066FED76E08AEDA0
:103B400096E00E94EF048091E2068093CE06809179
:103B5000E1068093CC068091E0068093CA068091AE
:103B60003807873008F449C1880F880F8B59809334
:103B7000DA066FED76E08AED96E00E94EF04809120
:103B8000E2068093CE068091E1068093CC06809178
:103B9000DA068E5F8093DA066FED76E08AED96E0C6
:103BA0000E94EF048091E2068093CA068091E106AC
:103BB00036C0803519F486E090E008C0813519F4EC
:103BC00087E090E003C090E0805490401092CC06D3
:103BD0000E94FE0F8093CE0690913807892F86545D
:103BE000823008F00AC1963419F40EE411E002C0E4
:103BF0000AE411E0C8010E94FE0F8093CE06C801BE
:103C000001960E94FE0F8093CC06C80102960E9486
:103C1000FE0F8093CA06C80103960E94FE0F809390
:103C2000CB06EBC01092CB061092CA061092CC06BF
:103C3000803819F48091400716C0813819F48091BA
:103C40004D0711C0823859F480913507909136079D
:103C5000892F99278093CC068091350704C083383B
:103C600029F48091A4018093CE062FC08438C9F432
:103C7000F8948091EA069091EB06A091EC06B09141
:103C8000ED0689839A83AB83BC8378948981809382
:103C9000CE068A818093CC068B818093CA068C8164
:103CA00012C0853891F40E943F3C6D837E838F83E0
:103CB00098878D818093CE068E818093CC068F81EC
:103CC0008093CA0688858093CB06809138078F3F02
:103CD00009F093C08091C1018EC0813009F074C099
:103CE0001092CB061092CA061092CC06809138072B
:103CF000882319F48091D10515C08130A9F0823054
:103D000019F48091B2060EC0833019F48091CD056C
:103D100009C0843019F48091CC0504C0853021F4A9
:103D20008091CE058093CE0680913807863039F495
:103D30008091D0058093CC068091CF055CC0873000
:103D400039F48091C9058093CC068091C80553C091
:103D5000883039F48091CB058093CC068091CA05D8
:103D60004AC0893079F48091B6068093CB06809161
:103D7000B5068093CA068091B4068093CC068091E4
:103D8000B30639C08A3079F48091BA068093CB06A5
:103D90008091B9068093CA068091B8068093CC06BC
:103DA0008091B70628C08B3041F58091C70580937C
:103DB000CB068091C6058093CA068091C505809385
:103DC000CC068091C40517C08230B9F4E091380761
:103DD000E83398F4F0E0EE0FFF1FEE0FFF1FEE52F6
:103DE000FA4F83818093CB0682818093CA068181BA
:103DF0008093CC0680818093CE0680915A078823D9
:103E000039F18091CB06809344078091CA06809354
:103E100043078091CC06809342078091CE06809321
:103E200041078091410790914207A0914307B091CB
:103E300044072091C2013091C3010097A105B1054B
:103E400011F4286001C0277F3093C3012093C20181
:103E500028960FB6F894DEBF0FBECDBFDF91CF918D
:103E60001F910F910895EF92FF920F931F93CF939D
:103E7000DF9380913907882309F024C180913807A6
:103E800087FDEEC0803458F5863061F42091CE066F
:103E9000207F6091CA066F7C60624091CC068EE7FD
:103EA0000E94D30500913807073008F4BBC110E029
:103EB000000F111F000F111F2091CE064091CC065C
:103EC00060E0802F8C590E94D3052091CA06409152
:103ED000CB0660E0802F8A590E94D305A3C18934A4
:103EE00009F58091B7019091B80124E0823D9207D5
:103EF00031F41092CC0681E08093CE060CC0815E36
:103F0000904129F41092CC061092CE0604C084E0B1
:103F10008093340787C16091CE0689E090E00E94CB
:103F2000061080C1803519F4C6E0D0E015C0813597
:103F300029F0C82FD0E0C054D0400EC08091CE06EA
:103F400080FD08C087E090E00E94FE0F80FF02C065
:103F50000E944830C7E0D0E080913807873419F4D8
:103F6000CAE4D1E004C0863411F4CEE4D1E0865432
:103F7000823090F46091CB06CE0103960E94061029
:103F80006091CA06CE0102960E9406106091CC068E
:103F9000CE0101960E9406106091CE06CE010E94CD
:103FA000061080913807873411F0853449F58AE48A
:103FB00091E00E94FE0F80932E078BE491E00E9417
:103FC000FE0F80932F078CE491E00E94FE0F8093F8
:103FD00030078DE491E00E94FE0F80933107E0905E
:103FE0002E07F0902F07009130071091310785E0E0
:103FF00090E00E94FE0FB801A70190E00E94933468
:10400000809138078634C1F48EE491E00E94FE0F5F
:104010008093E6068FE491E00E94FE0F8093E7060E
:1040200080E591E00E94FE0F8093E80681E591E033
:104030000E94FE0F8093E90680913807823421F4B4
:104040008091CE060E94283780913807833409F08A
:10405000E9C08091CE0682958F7080935F01E2C0A7
:10406000833829F48091CE068093A40121C084383E
:1040700099F4F8948091B9019091BA01A091BB0193
:10408000B091BC018093EA069093EB06A093EC06F6
:10409000B093ED0678940CC0853851F46091B90165
:1040A0007091BA018091BB019091BC010E94443C87
:1040B000809138078F3F09F0B5C08091CE0680937C
:1040C000C101B0C0813009F094C0809138078823C5
:1040D00029F48091CE068093D105A4C0813009F4E3
:1040E0004FC0823029F48091CE068093B2069AC0E8
:1040F000833029F48091CE068093CD0593C084301F
:1041000029F48091CE068093CC058CC0853029F4AB
:104110008091CE068093CE0585C0863079F480915B
:10412000CC0690E0982F88272091CE0630E0822B95
:10413000932B9093D0058093CF0574C0873079F48A
:104140008091CC0690E0982F88272091CE0630E011
:10415000822B932B9093C9058093C80563C0883048
:1041600079F48091CC0690E0982F88272091CE0694
:1041700030E0822B932B9093CB058093CA0552C0DD
:10418000893089F48091B9019091BA01A091BB0165
:10419000B091BC018093B3069093B406A093B5068A
:1041A000B093B6063FC08A3089F48091B9019091EE
:1041B000BA01A091BB01B091BC018093B706909366
:1041C000B806A093B906B093BA062CC08B3051F54F
:1041D0008091B9019091BA01A091BB01B091BC014D
:1041E0008093C4059093C505A093C605B093C705F9
:1041F00019C08230B9F4E0913807E83398F4F0E060
:10420000EE0FFF1FEE0FFF1FEE52FA4F8091CB060D
:1042100083838091CA0682838091CC0681838091BA
:10422000CE068083DF91CF911F910F91FF90EF9089
:104230000895309144073093CB0620914307209393
:10424000CA06909142079093CC06809141078093D3
:10425000CE069093B8018093B7013093BC012093B0
:10426000BB019093BA018093B9010E94331F089556
:104270000F931F93CF93DF93E0913807E7FD08C0BA
:10428000EF3008F0B9C0F0E0E059FE4FE49101C012
:10429000EF77E0933807909138079034C8F4E92F0E
:1042A000F0E0009139079F3040F4EE0FFF1F0295B8
:1042B000000F007E802F8E2B08C0EB5AFE4F84919A
:1042C000880F0295000F007E802B0E94350B94C052
:1042D0009B34E1F480913907C82FD0E0CC0FDD1F6B
:1042E000CE01865A9E4F0E94FE0FC15FD84F888331
:1042F00080913907C82FD0E0CC0FDD1FCE01855A41
:104300009E4F0E94FE0FC15FD84F1DC09C34E9F440
:1043100080913907C82FD0E0CC0FDD1FCE01805A25
:104320009E4F0E94FE0FCF50D94F8883809139074E
:10433000C82FD0E0CC0FDD1FCE018F599E4F0E94B9
:10434000FE0FCF50D94F898357C09335E1F4809148
:104350003907C82FD0E0CC0FDD1FCE018A599E4F00
:104360000E94FE0FC95ADE4F888380913907C82FFB
:10437000D0E0CC0FDD1FCE0189599E4F0E94FE0F69
:10438000C95ADE4FE0CF892F8155823020F483E077
:104390008093340731C0009139079D3459F410E0FF
:1043A000C80183509C4F0E94FE0F0A5E184FF8010F
:1043B000808322C0C02FD0E0C05CD04083E0989FB3
:1043C000C0011124C80FD91FCE0140960E94FE0FD4
:1043D0008093CE06682F8C2F0E948C108091380716
:1043E000853451F4CE010D960E94FE0F682F9E0178
:1043F0002350822F0E948C10DF91CF911F910F913B
:1044000008951F93CF93DF93E0913807E7FD08C02D
:10441000EF3008F0B3C0F0E0E059FE4FE49101C086
:10442000EF77E0933807209138072034D0F4E22F5B
:10443000F0E0909139072F3040F4EE0FFF1F929576
:10444000990F907E892F8E2B08C0EB5AFE4F8491D6
:10445000880F9295990F907E892B0E94EB0A182F56
:1044600088C02B34C9F48091390790E0880F991FD8
:10447000FC01E15FF84F6081865A9E4F0E94061052
:104480008091390790E0880F991FFC01E15FF84F98
:104490006181855A9E4F1AC02C34D9F48091390716
:1044A00090E0880F991FFC01EF50F94F6081805A0E
:1044B0009E4F0E9406108091390790E0880F991F47
:1044C000FC01EF50F94F61818F599E4F0E940610F9
:1044D00055C02335C9F48091390790E0880F991FA2
:1044E000FC01E95AFE4F60818A599E4F0E940610D6
:1044F0008091390790E0880F991FFC01E95AFE4F1F
:10450000618189599E4FE2CF2D3451F48091390752
:1045100090E0FC01EA5EF84F608183509C4FD6CF5B
:10452000822F8155823010F483E026C080913907B4
:10453000C82FD0E0C05CD04083E0289FC001112488
:10454000C80FD91F8C2F0E948510682FCE0140966E
:104550000E940610182F80913807853451F49E016F
:104560002350822F0E948510682FCE010D960E9445
:104570000610123019F485E080933407DF91CF9153
:104580001F910895DF92EF92FF920F931F93CF93A5
:10459000DF93CDB7DEB726970FB6F894DEBF0FBE18
:1045A000CDBFE0913807E7FD08C0EF3008F007C243
:1045B000F0E0E059FE4FE49101C0EF77E093380757
:1045C000209138072B3108F0B3C0233041F4E0913B
:1045D0003907F0E0EE0FFF1FE45AF84F09C026300C
:1045E00061F4E0913907F0E0EE0FFF1FEA5BF84F4E
:1045F00081818093CC06808190C090913907E22F11
:10460000F0E0293058F5EE0FFF1F9295990F907E3C
:104610009E2B91609093DA066FED76E08AED96E03E
:104620000E94EF048091E0068093CA069091E10613
:104630009093CC068091E2068093CE068091380755
:10464000843008F46CC093FF6AC0906F9093CC06DE
:104650008FEF8093CA068093CB0661C0EB5AFE4F62
:104660008491880F9295990F907E982B91609093EA
:10467000DA066FED76E08AED96E00E94EF041E8286
:104680008091E0068D838091E1068C838091E20623
:104690008B832B813C814D815E81E09138078E2F89
:1046A00090E0FC01ED5BFE4FE49104C05595479509
:1046B00037952795EA95D2F72B833C834D835E830C
:1046C000815D9E4FEE24FF24870160E070E0FC01D5
:1046D000D4900FC081E090E0A0E0B0E004C0880F6B
:1046E000991FAA1FBB1FEA95D2F7E82AF92A0A2BBD
:1046F0001B2BE62F6F5F7F4FED1560F3E222F32255
:1047000004231523EB82FC820D831E838D8180930D
:10471000CA068C818093CC068B818093CE068091D3
:10472000CA0687FF02C08FEF1DC11092CB061CC1C5
:104730002E3108F03FC01092CB061092CA0610929C
:10474000CC061092CE068DE78093DA066FED76E008
:104750008AED96E00E94EF04809138078B3199F43E
:1047600080913907880F22E030E002C0220F331F0A
:104770008A95E2F78091E20690E028233923232BE3
:1047800009F4F2C015C08C3119F48091E20605C01D
:104790008D3109F0E9C08091DF0690E02091390762
:1047A000220F02C0959587952A95E2F780FFDCC01D
:1047B00081E098C0203408F4D7C0203608F095C0B6
:1047C00010913907105C83E0289FC0011124180F55
:1047D000253431F4812F83500E9485108093CC06BC
:1047E000812F0E9485108093CE06809138078B34EC
:1047F000A9F4E0913907F0E0EE0FFF1FE15FF84FF9
:1048000091819093CC0680818093CE0697FF1FC044
:104810008FEF8093CB068093CA0619C08C3441F485
:10482000E0913907F0E0EE0FFF1FEF50F94F09C09C
:10483000833569F4E0913907F0E0EE0FFF1FE95A84
:10484000FE4F81818093CC0680818093CE0680913B
:1048500038078D3431F4E0913907F0E0EA5EF84F23
:104860000FC08E3431F4E0913907F0E0ED51F94F8B
:1048700007C0803541F4E0913907F0E0E450F94F8A
:1048800080818093CE06809138078135A1F4809194
:1048900039070E94CA386B837C838D839E838E8107
:1048A0008093CB068D818093CA068C818093CC0641
:1048B0008B818093CE0680913807873419F080343D
:1048C00009F052C09091CE0684E6989FC001112451
:1048D00061E170E00E94C33C7A8369838A8180939E
:1048E000CC0689818093CE063FC02236C1F4109257
:1048F000CC06E0913907F0E0E35CF84F808181FF5E
:1049000004C081E08093CE0602C01092CE06E091F2
:104910003907F0E0E35CF84F80818D7F80838091E0
:1049200038078336C1F41092CC06E0913907F0E0E5
:10493000E35CF84F808182FF04C081E08093CE0663
:1049400002C01092CE06E0913907F0E0E35CF84F28
:1049500080818B7F80838091CC0687FF05C08FEF9D
:104960008093CA068093CB0680915A07882339F139
:104970008091CB06809344078091CA0680934307B9
:104980008091CC06809342078091CE0680934107A8
:104990008091410790914207A0914307B09144074D
:1049A0002091C2013091C3010097A105B10511F416
:1049B000286001C0277F3093C3012093C20126964F
:1049C0000FB6F894DEBF0FBECDBFDF91CF911F9120
:1049D0000F91FF90EF90DF9008950F931F93CF9367
:1049E000DF93982FC82FDD27C7FDD095FE01E65C29
:1049F000F84F8081882319F480E090E01EC0108277
:104A00008E01000F111FF801EA5BF84F6081718180
:104A1000892F0E947008045A184F25E0CC0FDD1F23
:104A20002A95E1F7F8012081418160E0FE01E6600E
:104A30008E2F0E94D30581E090E0DF91CF911F91EE
:104A40000F910895CF93DF93CDB7DEB722970FB6BE
:104A5000F894DEBF0FBECDBF90913907E92FF0E08B
:104A6000E65CF84F8081813019F4892F0E94ED2493
:104A70008091B7019091B801909581959F4F9A834D
:104A8000898362E0809139070E94FC088091390790
:104A90008295880F807E29814A8160E088600E942B
:104AA000D305809139078295880F807E2FEF47E0EC
:104AB00060E086600E94D305E0913907F0E0E65C93
:104AC000F84F82E0808322960FB6F894DEBF0FBEC7
:104AD000CDBFDF91CF91089590913907E92FF0E094
:104AE000E65CF84F8081813019F4892F0E94ED2413
:104AF00062E0809139070E94FC0880913907829515
:104B0000880F807E2091CE064091CC0660E08860C0
:104B10000E94D305809139078295880F807E2FEF00
:104B200047E060E086600E94D305E0913907F0E03D
:104B3000E65CF84F82E080830895DF92EF92FF9267
:104B40000F931F93CF93DF93CDB7DEB724970FB6A4
:104B5000F894DEBF0FBECDBFD62E082F10E0C801DF
:104B6000E5E0880F991FEA95E1F782600E9441080D
:104B70009B01AC01DD2069F17801EE0CFF1CE00E19
:104B8000F11E8BE192E0E80EF91E89E0D89EC0018B
:104B90001124E80EF91E9FECE91692E0F90624F0C4
:104BA00081E08093340720C029833A834B835C8360
:104BB0006B81C70102960E940610FE013196618149
:104BC000C70101960E9406106981C7010E94061064
:104BD0000BC0000F111F000F111F025B184FF801CF
:104BE000208331834283538324960FB6F894DEBF2B
:104BF0000FBECDBFDF91CF911F910F91FF90EF902E
:104C0000DF9008951F931091380780913907833002
:104C100010F4612F30C0843041F4612F80E00E9495
:104C20009D25612F81E00E949D2580913907853067
:104C300041F4612F81E00E949D25612F82E00E9456
:104C40009D2580913907863041F4612F80E00E94D4
:104C50009D25612F82E00E949D2580913907873034
:104C600061F4612F80E00E949D25612F81E00E9408
:104C70009D25612F82E00E949D251F910895CF926E
:104C8000DF92EF92FF920F931F93182F062F8295BA
:104C9000880F807E82600E9441086B017C01602F3A
:104CA000812F0E94E4176C157D058E059F0529F460
:104CB00060E070E080E090E010C0C616D706E8061D
:104CC000F9062CF46C197D098E099F0906C0C61AD5
:104CD000D70AE80AF90AC701B6011F910F91FF90A0
:104CE000EF90DF90CF9008950F931F93182F062F0A
:104CF00060E00E94FC08602F812F0E94E417AB0146
:104D0000BC01812F8295880F807E0E9418091F9117
:104D10000F9108954F925F926F927F928F929F9220
:104D2000AF92BF92CF92DF92EF92FF920F931F93B9
:104D3000CF93DF93CDB7DEB728970FB6F894DEBFD9
:104D40000FBECDBF4091CB0648872091CA062F8366
:104D50003091CC063E838091CE068D83E09138075A
:104D6000E7FD08C0EF3008F096C1F0E0E059FE4FD3
:104D7000E49101C0EF77E0933807E0913807E7341A
:104D800011F0E03479F48091B7019091B80153E0CB
:104D9000880F991F5A95E1F76FE270E00E94D73CA7
:104DA0006093CE06E03408F0E8C0E930B0F5E630B4
:104DB00081F46091B7017091B801809139070E9428
:104DC0007008E0913907F0E0EE0FFF1FEA5BF84F43
:104DD000DDC02093DB063093DC068091CE06809305
:104DE000DD06EE0F809139078295880F807E8E2B2D
:104DF0008093DA066FED76E08AED96E00E94EF048C
:104E000080913807833009F03AC1E0913907F0E02A
:104E1000EE0FFF1FE45AF84FB9C0E031E9F480917A
:104E200039078295880F807E81618093DA066FED65
:104E300076E08AED96E00E94EF0480913907829532
:104E4000880F807E80618093DA069091CE069F70F5
:104E50008091E006807F1FC090913907E13169F5AC
:104E60009295990F907E91619093DA066FED76E0BE
:104E70008AED96E00E94EF04809139078295880FB1
:104E8000807E80618093DA069091CE069295907F25
:104E90008091E0068F70982B9093DB068091E1065D
:104EA0008093DC068091E2068093DD066FED76E06C
:104EB0008AED96E00E94EF04E2C01C822B833A83C5
:104EC0008091CE068983F0E0EB5AFE4FE491EE0F1D
:104ED000B92EB294BB0C90EEB922BE2A8B2D0E9443
:104EE0004108AB01BC01E09138078E2F90E0FC0136
:104EF000ED5BFE4FE49101E010E020E030E004C003
:104F0000000F111F221F331FEA95D2F7C980DA80E4
:104F1000EB80FC8044245524815D9E4FFC01A490CD
:104F200025C03601470104C095948794779467940F
:104F30008A95D2F7D401C30181709070892B29F032
:104F4000402B512B622B732B0AC0D901C8018095CD
:104F50009095A095B095482359236A237B23000F91
:104F6000111F221F331F0894411C511C842D4A1409
:104F7000C0F28B2D0E94180982C0EB3471F4E091CD
:104F80003907F0E0EE0FFF1FE15FF84F8091B701A6
:104F90009091B8019183808372C0EC3441F4E09128
:104FA0003907F0E0EE0FFF1FEF50F94FEFCFE33579
:104FB00041F4E0913907F0E0EE0FFF1FE95AFE4F90
:104FC000E5CFED3449F4E0913907F0E0EA5EF84FBF
:104FD0008091CE06808353C0E13579F44C832B83D6
:104FE0003A838091CE06898349815A816B817C8185
:104FF000809139070E94073842C0E235C1F44C83E2
:105000002B833A838091CE06898369817A818B8153
:105010009C81462F4F71F5E095958795779567951B
:10502000FA95D1F7809139070E942D3828C0E036D3
:1050300030F510913907105C83E0E89FC00111241E
:10504000180FE53429F4632F812F83500E948C10B0
:105050006091CE06812F0E948C10809139078B5E63
:105060000E948510682F809139070E94CD0F809192
:105070003807873411F0803411F41092CC068885FB
:105080008093CB068F818093CA068E818093CC0655
:105090008D818093CE0628960FB6F894DEBF0FBEA2
:1050A000CDBFDF91CF911F910F91FF90EF90DF90D7
:1050B000CF90BF90AF909F908F907F906F905F90B8
:1050C0004F900895309144073093CB0620914307C9
:1050D0002093CA06909142079093CC068091410795
:1050E0008093CE069093B8018093B7013093BC01B2
:1050F0002093BB019093BA018093B9010E948A2644
:1051000008951092CB061092CA061092CC06809198
:105110003907882331F580913807883018F40E94C8
:10512000980F1DC08A30A0F40E94CA0F90E0209111
:10513000380730E02850304002C0959587952A9571
:10514000E2F780FF02C081E00AC01092CE0609C0DB
:1051500083B390E096958795969587958170809317
:10516000CE0680913907813081F4E0913807F0E074
:10517000EE0FFF1FE150F94F208131818181837053
:105180008093CC062093CE0608C0823031F4809103
:1051900038070E94BC0F8093CE0680915A0788235F
:1051A00059F18091CB06809344078091CA06809381
:1051B00043078091CC06809342078091CE0680936E
:1051C00041078091410790914207A0914307B09118
:1051D00044072091C2013091C3010097A105B10598
:1051E00031F428603093C3012093C2010895277FD2
:1051F0003093C3012093C201089580913907882319
:1052000039F46091CE06809138070E94A20F08956C
:10521000823071F48091CE0680FF05C080913807FE
:105220000E94900F0895809138070E94940F08956E
:105230008F3F21F56091CE0680E00E944C05609181
:10524000CC0681E00E944C056091CA0682E00E9473
:105250004C058091CE0682FF03C080E00E944E097B
:105260008091CC0682FF03C081E00E944E098091AC
:10527000CA0682FF03C082E00E944E0908950F9380
:105280001F93CF93DF93CDB7DEB72F970FB6F89468
:10529000DEBF0FBECDBF80913D079091BB06892B2D
:1052A00080933D0780913E079091BC06892B8093A7
:1052B0003E078091BD0690913F07892B80933F0761
:1052C00080911907882349F08091C2019091C30110
:1052D00091609093C3018093C2018091320780FF57
:1052E0000BC08091BD019091BE01009729F00197FC
:1052F0009093BE018093BD010E94F509282F8093F1
:10530000EB014091E9015091EA014130510519F05A
:10531000882309F4A1C03091DE06832F81508230AA
:1053200010F02230E1F58091E6069091E706A09119
:10533000E806B091E9068C839D83AE83BF831A8211
:105340001B822230C1F0313011F497E001C098E0A7
:10535000EFEAF1E0DE01189681918D9321E0E73BC1
:10536000F207D1F79983CE0101960E945A3588231E
:1053700009F47DC222C0EDE1F7E0DE0118968191CB
:105380008D9387E0E532F807D1F787E08983CE0176
:1053900001960E945A35882309F469C25AC0809147
:1053A0001507882319F4233091F40DC0233059F0E8
:1053B00068E08FEA91E00E9452378091E901909174
:1053C000EA018E7F50C268E08DE197E0F4CF8091D2
:1053D000F706882309F04BC280915E01213039F134
:1053E0004E7F5093EA014093E9018230A0F40EEA27
:1053F00011E0F80181918F010E94ED2FF1E0073B50
:105400001F07B9F780915E01813009F030C282E058
:1054100080935E012CC28EEA91E00E945E398091F9
:105420005E01833009F023C210925E0120C28823FE
:1054300061F40CE117E0F80181918F010E94ED2FDA
:10544000F7E005321F0729F0F6CF8EEA91E00E94BF
:105450005E391092EB010BC21092C80180915E017F
:10546000882331F482E697E00E941C07813051F0D6
:1054700080915E018823A1F182E697E00E94F439D1
:10548000813071F581E08093C8018091620780933B
:105490006E0780916307809338078091640780933B
:1054A0003907809165078093CB06809166078093CA
:1054B000CA06809167078093CC0680916807809325
:1054C000CE0680914007882319F481E090E053C014
:1054D00020E030E0833011F421E030E0C9014BC01E
:1054E0008091320782FF23C080914007813009F00C
:1054F00044C090919201913009F03FC083E08093C5
:10550000C80187E180936E0710923807109239071F
:105510001092CB061092CA068091DF018093CC06D0
:105520008091E0018093CE0690935A0726C00E9496
:105530003F17882311F182E08093C8018091A50173
:1055400080936E078091A601809338078091A70110
:10555000809339078091A8018093CB068091A9019F
:105560008093CA068091AA018093CC068091AB01FA
:105570008093CE0681E080935A078091C8018823EA
:1055800009F475C182E090E00E94FE0F382F8093ED
:105590004C072091CC062093B8019091CE069093B1
:1055A000B7018091CB068093BC018091CA0680939D
:1055B000BB012093BA019093B901109234079091E6
:1055C0006E07892F8854883310F09E3870F08091D0
:1055D000C801813011F4923F41F082E0809334079A
:1055E0008091A40181608093A4018091C8018130E1
:1055F00091F4E2E6F7E08191380F27E0E936F2070F
:10560000D1F730934C07809169073817C9F081E0D2
:105610008093340715C0823099F4E5EAF1E0819176
:10562000380F81E0EC3AF807D1F730934C078091BE
:10563000AC01381729F08091A40182608093A40105
:105640001092C00180913407882309F095C08091A1
:105650004D07882311F097FF50C0923F21F40E941C
:10566000A81682E087C0E92FF0E097FF05C0EE0F93
:10567000FF1FE051F04004C0EE0FFF1FE05AFF4F44
:105680000190F081E02D84E6809334078091EC0155
:10569000882311F0099503C08FEF80933407609140
:1056A000DD017091DE016115710509F465C080911D
:1056B0004007813009F060C08091C801823009F054
:1056C0005BC0409135075091360720E030E00FC0B5
:1056D0002F5F3F4FEE0FFF1FE753FE4F80819181F9
:1056E0004817590721F485E08093400745C0E22F11
:1056F000F0E0E617F70760F33FC08091C401909196
:10570000C501E7E08F3F9E07A0F562E677E00E94C3
:10571000FA30882371F561EE71E08091C4019091B7
:10572000C5010E94C43085E68093340720E030E054
:10573000F901EF51FE4FD901AE59B84F90818C91CC
:10574000981721F087E08093340705C02F5F3F4F03
:105750002830310569F780913407853669F48091E6
:10576000C4019091C50101969093C5018093C40135
:1057700003C087E0809334078091C801813009F02D
:1057800076C08CE090E00E94FE0F182F82E090E03F
:105790000E94FE0F282F809337078091C001882335
:1057A000C9F590916E07963031F48091CA06880F42
:1057B000880B8093CB061093AE012093AF018091AC
:1057C00034078093B0019093B1018091CB06809310
:1057D000B2018091CA068093B3018091CC06809378
:1057E000B4018091CE068093B5018091150788237E
:1057F00039F010924C0790914C07EFEAF1E003C0AA
:1058000010934C07F8CF8191980F21E0E63BF20707
:10581000D1F70FC0813089F41093AE0110924C077C
:10582000EEEAF1E090E08191980F81E0E63BF80725
:10583000D1F790934C079093B6018BE090E00E94D3
:10584000FE0F8093F7068091C101882351F080916B
:105850006E07863031F08A3021F08F3011F08F31B1
:1058600031F481E090E09093EA018093E9012F9672
:105870000FB6F894DEBF0FBECDBFDF91CF911F9161
:105880000F9108959F92AF92BF92CF92DF92EF92C5
:10589000FF920F931F93CF93DF93CDB7DEB722977D
:1058A0000FB6F894DEBF0FBECDBF6C017B01042F95
:1058B0006115710509F499C0009709F496C068173D
:1058C000790709F492C0142F1295110F107EA6E0EB
:1058D0009A2E912A892D0E9427089A838983812FE5
:1058E0008C600E9427085C0180E0D7FC07C0EE0CAA
:1058F000FF1CCC0CDD1C8F5F8F30B9F7E114F10475
:1059000019F471E0E72EF12C40E050E001C079017C
:10591000142F4F5F5F4FC70180709E7F97013695B0
:105920002795892BA1F7C9018C0D9D1DB7010E94F8
:10593000C33CFB01672B11F4E1E0F0E089819A811F
:1059400054E0880F991F5A95E1F7BF010E94C33CAC
:105950009B01C50144E0880F991F4A95E1F7BF01FB
:105960000E94C33C412F50E0153090F484E090E059
:10597000841B950B082E02C0369527950A94E2F7F2
:105980003A83298302C0769567958A95E2F70FC01E
:10599000CA010497082E02C0220F331F0A94E2F7AF
:1059A0003A83298302C0660F771F8A95E2F78981BF
:1059B0009A81892B21F481E090E09A838983611593
:1059C000710511F461E070E0749718F4802F0E9463
:1059D000700829814A8160E0892D0E94D305E02F5B
:1059E000F0E0E65CF84F81E0808322960FB6F894F1
:1059F000DEBF0FBECDBFDF91CF911F910F91FF9002
:105A0000EF90DF90CF90BF90AF909F9008950F934D
:105A10001F93CF93DF93CDB7DEB762970FB6F8949D
:105A2000DEBF0FBECDBF082F162F8430C1F480E03B
:105A30000E94ED2481E00E94ED24612F80E00E940D
:105A40003F266F83788789879A87612F81E00E943C
:105A50003F266B877C878D879E87198A3FC085305C
:105A600041F481E00E94ED2482E00E94ED24198639
:105A700025C0863081F480E00E94ED2482E00E94FF
:105A8000ED24612F80E00E943F266F83788789870D
:105A90009A871D861BC0873009F580E00E94ED249F
:105AA00081E00E94ED2482E00E94ED24612F80E0DD
:105AB0000E943F266F83788789879A87612F81E0CC
:105AC0000E943F266B877C878D879E87612F82E0AF
:105AD0000E943F266F87788B898B9A8B99859923B3
:105AE00031F48D85882319F48989882369F09A8394
:105AF000FE013796818189838D858C838C858B838C
:105B000089898E8388890BC088858A838F81898360
:105B10008C858C838B858B8388898E838F858D8301
:105B2000043049F429813A818B819C818217930743
:105B3000D0F441E015C0053049F42B813C818D81C2
:105B40009E818217930758F041E00EC0063071F431
:105B500029813A818D819E818217930720F442E04A
:105B6000BC01C90133C040E0B90130C0073081F544
:105B700089819A812B813C81ED81FE81281739072B
:105B800068F4E817F907C0F441E0B9010E94422C1B
:105B90006D817E8142E089819A8118C0E217F30706
:105BA00058F440E0BC01C9010E94422C6D817E8105
:105BB00042E08B819C810AC040E0BC01CF010E9481
:105BC000422C6B817C8141E08D819E810E94422C20
:105BD00062960FB6F894DEBF0FBECDBFDF91CF91B6
:105BE0001F910F910895CF92DF92EF92FF920F9342
:105BF0001F93CF93DF93CDB7DEB724970FB6F894FA
:105C0000DEBF0FBECDBF80913807823008F04BC099
:105C100060E0809139070E94FC08809139070E945A
:105C2000ED246E010894C11CD11C8091CB068C839D
:105C30008091CA068B838091CC06F6018183809186
:105C4000CE06898380913807813009F5E980FA8092
:105C50000B811C81809139078295880F807E82603C
:105C60000E944108E60EF71E081F191FE982FA82FA
:105C70000B831C838C818093CB068B818093CA0617
:105C8000F60181818093CC0689818093CE0649817B
:105C90005A816B817C81809139078295880F807E43
:105CA0000E94180946C0823009F043C0E090CE0639
:105CB00080913907833030F40E94ED246E2D80915D
:105CC000390735C06E2D0E94072D80913907843029
:105CD00041F46E2D80E00E9474266E2D81E00E94BA
:105CE000742680913907853041F46E2D81E00E9441
:105CF00074266E2D82E00E947426809139078630CA
:105D000041F46E2D80E00E9474266E2D82E00E9488
:105D1000742680913907873061F46E2D80E00E94EF
:105D200074266E2D81E00E9474266E2D82E00E9402
:105D3000742624960FB6F894DEBF0FBECDBFDF9158
:105D4000CF911F910F91FF90EF90DF90CF9008952A
:105D5000CF92DF92EF92FF920F931F93CF93DF9337
:105D600010923607109235078FEF9FEF9093C7017F
:105D70008093C6018DE090E00E94FE0F813011F407
:105D80008093400716E4C12E17E0D12EBCE5EB2E20
:105D9000B7E0FB2EC0E0D0E0CE018295880F807E78
:105DA000182F8C600E942708F601819391936F0150
:105DB000812F86600E942708F701819391937F01CC
:105DC0002196C330D10541F702ED15E0CEE1D3E0D5
:105DD000CE010E94FE0FF8018383CE0101970E943D
:105DE000FE0FF8018283CE0102970E94FE0FF80198
:105DF0008183CE0103970E94FE0FF80180832496D1
:105E00000C5F1F4FF3E0CE3FDF0711F7ECEFFFE72A
:105E1000E491E73299F4EDEFFFE7E491E83171F4B2
:105E2000EEEFFFE7E491E83249F4EFEFFFE7E491AA
:105E3000E83121F481E08093EC0102C01092EC0182
:105E4000DF91CF911F910F91FF90EF90DF90CF9056
:105E500008951F920F920FB60F9211248F939F9364
:105E6000EF93FF938BB1887129F08091ED018062EF
:105E70008093ED01869B04C08CB180931F021AC0F1
:105E8000809109029CB1E82FF0E0E251FE4F90832F
:105E90008F5F809309028B3110F01092090290916C
:105EA000090280910A02981729F48091ED01806817
:105EB0008093ED01FF91EF919F918F910F900FBE15
:105EC0000F901F9018951F920F920FB60F921124EA
:105ED0008F939F93EF93FF9390911E0280911D02E9
:105EE000981781F0969AE92FF0E0E55FFD4F8081E9
:105EF0008CB9892F8F5F80931E02823120F010921F
:105F00001E0201C05598FF91EF919F918F910F90C4
:105F10000FBE0F901F9018951F920F920FB60F9201
:105F200011248F939F9390911E0280911D029817C8
:105F300009F496989F918F910F900FBE0F901F902C
:105F40001895982F8091090280930A0280911E0271
:105F500080931D021092ED012091D306283019F490
:105F6000EEE7F1E002C0E7E8F1E0849189B988ED5D
:105F70008AB9992369F0993058F4E92FF0E0283074
:105F800019F4E258FE4F02C0E957FE4F849189B9D7
:105F900008958091ED0181FF02C01092ED018BB157
:105FA000887129F08091ED0180628093ED018091EC
:105FB000ED0182608093ED01807F19F08FEF9FEFFC
:105FC000089520E030E090910A028091090298172C
:105FD00011F021E030E0C9010895969A90911D02D8
:105FE000E92FF0E0E55FFD4F80839F5F90931D02F6
:105FF000923110F010921D0290911D0280911E02AC
:10600000981729F48091ED0180648093ED01559AF1
:106010000895DC0190910A0280910902981719F401
:1060200080E090E00895E92FF0E0E251FE4F80819A
:106030008C93892F8F5F80930A028B3118F481E053
:1060400090E0089510920A0281E090E00895209176
:106050001D022E5F30911E02223138F080E090E068
:10606000332349F481E090E0089580E090E0231725
:1060700011F481E090E0089520E030E090911E025C
:1060800080911D02981711F421E030E0C9010895B4
:10609000EF92FF920F931F93CF93DF93CDB7DEB7AD
:1060A00022970FB6F894DEBF0FBECDBF1A821982B9
:1060B0007E010894E11CF11C46C08BB78F7B8BBF1F
:1060C000C49886E00E94A810C49A8BB780648BBFE6
:1060D0008BB78F7B8BBFC49882E00E94A810F7011A
:1060E00081810E94A81089810E94A81000E010E020
:1060F00089819A81800F911F885F9F4340F480E0DF
:106100000E94A8100F5F1F4F0034110589F7C49A31
:106110008BB780648BBF00E010E01CC0C49A8BB7C3
:1061200080648BBF0AC0C49A8BB780648BBF0F5F3B
:106130001F4F2EE2003E120769F489819A81805C2C
:106140009F4F9A83898389819A818050904408F473
:10615000B4CF0DC08BB78F7B8BBFC49885E00E94F6
:10616000A81080E00E94A81080FDDDCFD7CF229636
:106170000FB6F894DEBF0FBECDBFDF91CF911F9158
:106180000F91FF90EF900895EF92FF920F931F935E
:10619000CF93DF937B018C0193E0000F111F9A9541
:1061A000E1F78BB78F7B8BBFC49883E00E94A81068
:1061B000812F99270E94A810802F0E94A810C0E06C
:1061C000D0E087010C0F1D1F80E00E94A810F8018D
:1061D00080832196C830D105A1F7C49A8BB780641B
:1061E0008BBF80E090E0DF91CF911F910F91FF90E6
:1061F000EF900895EF92FF920F931F93CF93DF9349
:106200007B018C0133E0000F111F3A95E1F78BB74A
:106210008F7B8BBFC49886E00E94A810C49A8BB76E
:1062200080648BBF8BB78F7B8BBFC49882E00E944A
:10623000A810812F99270E94A810802F0E94A810D3
:10624000C0E0D0E0F701EC0FFD1F80810E94A81094
:106250002196C830D105B1F7C49A8BB780648BBF43
:10626000C0E0D0E013C0C49A8BB780648BBF80E0DD
:1062700090E019C0C49A8BB780648BBF21968EE2E0
:10628000C03ED80719F48FEF9FEF0DC08BB78F7BFF
:106290008BBFC49885E00E94A81080E00E94A810DF
:1062A00080FDE8CFE0CFDF91CF911F910F91FF905C
:1062B000EF9008959091E20696959093E206809172
:1062C000E10680FF03C090689093E2069091E1069A
:1062D00096959093E1068091E00680FF03C0906858
:1062E0009093E1068091E00686958093E00686FF14
:1062F00003C080688093E0060895E82FF0E0EE0F79
:10630000FF1FEF5CFD4F80819181009719F001978D
:10631000918380830895BF92CF92DF92EF92FF9294
:106320000F931F93CF93DF93082FC82EDD24F60120
:10633000E251F94F108123E0B22EB80E8B2D0E944E
:106340008510E601CC0FDD1F843098F48DE70E94A4
:106350001A0822E030E00C2E02C0220F331F0A94EC
:10636000E2F7F82EF2228DE70E941A0821E030E0D1
:1063700012C08DE70E941A0821E030E00C2E02C006
:10638000220F331F0A94E2F7F82EF2228DE70E94C3
:106390001A0822E030E002C0220F331FCA95E2F74C
:1063A0008223E02EE294EE0CB0EEEB22113019F5D0
:1063B000F601EE0FFF1FEF5CFD4F1182108285E1A9
:1063C000E82AE092DA066FED76E08AED96E00E9428
:1063D000EF04F601E25DFD4F8091E106808362E00B
:1063E000802F0E94FC088B2D0E948510823008F4BB
:1063F000B8C112E0B7C1123051F4802F8A5F0E94F9
:106400008510682F802F0E94760913E0ABC11330EE
:1064100021F4882309F0A5C1A5C1143051F4802FBF
:106420008A5F0E948510682F802F0E94590915E00D
:1064300099C1153089F4FF2009F494C1802F0E947E
:106440004E09F601EE0FFF1FEF5CFD4F8EE190E06D
:106450009183808316E086C11630A1F4F601EE0F19
:10646000FF1FEF5CFD4F80819181892B09F07AC17C
:10647000802F875F0E948510682F802F0E947609E9
:1064800017E070C11730D9F4FF2009F06BC122E08A
:1064900043E060E08E2D84610E94D30520E040E05F
:1064A00060E08E2D8C610E94D305802F875F0E9453
:1064B0008510682F802F0E94590918E053C11830A9
:1064C00011F5FF2009F44EC1802F0E944E098E2D38
:1064D0008D618093DA066FED76E08AED96E00E949A
:1064E000EF042091E2064091E1066091E0068E2DD6
:1064F0000E94D30520E043E060E08E2D84610E947D
:10650000D30519E02FC1193009F041C08DE7809300
:10651000DA066FED76E08AED96E00E94EF04809156
:10652000DF0690E09601220F331F02C095958795F4
:106530002A95E2F780FF16C18B2D0E948510182F37
:1065400062E0802F0E94FC08802F0E944E0920E00C
:1065500040E060E08E2D0E94D30520E040E060E046
:106560008E2D82600E94D305133039F08091200275
:1065700090912102892B09F473C0802F875F0E94BC
:106580008510682F802F0E9459091AE0EBC01A303D
:1065900061F4FF2009F4E6C020E040E060E08E2DC9
:1065A0008C610E94D3051BE0DDC01B3009F05AC08E
:1065B000FF2009F0D7C0802F0E944E098E2D8D61DB
:1065C0008093DA066FED76E08AED96E00E94EF04A4
:1065D0000E945A312091E2064091E1066091E00666
:1065E0008E2D0E94D30520E043E060E08E2D846173
:1065F0000E94D3051091E20610951093E2060091D7
:10660000E10600950093E106F090E006F094F09228
:10661000E0060E945A318091E206810F8093E206E3
:10662000882329F48091E1068F5F8093E1068091B1
:10663000E106800F8093E106882329F48091E0062B
:106640008F5F8093E0066091E0066F0D6093E00637
:106650002091E2064091E1068E2D8A610E94D305C9
:106660001EE080C01E3009F06EC08091DF0690E011
:106670009601220F331F02C0959587952A95E2F760
:1066800080FF70C062E0802F0E94FC08802F0E9473
:106690004E098B2D0E948510833031F080912002AD
:1066A00090912102892B91F01092DF061092E00662
:1066B0001092E106F601EE0FFF1FEE0FFF1FEE5DD9
:1066C000FD4F108211821282138203C08E2D0E9410
:1066D000350B2091E2064091E1066091E0068E2D97
:1066E0000E94D3051E2D12602091E2064091E10622
:1066F0006091E006812F0E94D30520E040E060E039
:106700008E2D0E94D30520E040E060E0812F0E94A2
:10671000D305F601E25DFD4F20E0408160E08E2D63
:1067200084610E94D305F601EE0FFF1FE45AF84F73
:1067300040815181662757FD6095762F8E2D8660AA
:106740000E9418090CC01F3069F4F601E25DFD4F8C
:1067500022E0408160E08E2D84610E94D30510E02C
:1067600001C014E0EEEEF6E0CE0EDF1EF60110835F
:10677000DF91CF911F910F91FF90EF90DF90CF901D
:10678000BF900895AC018091A704882319F480E09C
:1067900090E008958BB78F7B8BBF909138028091EA
:1067A0003702981711F490E01EC020913802822F12
:1067B00090E0FC0134E0EE0FFF1F3A95E1F7E81B93
:1067C000F90BDA01E959FC4F8FE001900D928150ED
:1067D000E1F72F5F2093380280913802843111F461
:1067E0001092380291E08BB780648BBF892F90E0C4
:1067F00008950F931F93CF93DF93DA9895E09093CA
:106800009304809394046093950440939604C0E0AD
:10681000D0E08E010D561B4FF80180810E94A81018
:10682000F80180832196C430D10599F7DA9ADF9177
:10683000CF911F910F910895EF92FF920F931F93A5
:10684000CF93DF93DA9892E090939304809394042B
:10685000EE24FF24C62FD0E0229609C08C010D56ED
:106860001B4FF80180810E94A810F80180838E2DB3
:1068700090E00894E11CF11C8C179D077CF3DA9AD8
:10688000DF91CF911F910F91FF90EF9008950F939B
:106890001F93CF93DF93DA9892E0909393048093C1
:1068A000940460939504C0E0D0E08E010D561B4F18
:1068B000F80180810E94A810F80180832196C330DE
:1068C000D10599F7DA9ADF91CF911F910F91089531
:1068D000EF92FF920F931F93CF93DF93DA9893E099
:1068E0009093930480939404EE24FF24C62FD0E069
:1068F000229609C08C010D561B4FF80180810E9421
:10690000A810F80180838E2D90E00894E11CF11C02
:106910008C179D077CF3DA9ADF91CF911F910F912D
:10692000FF90EF900895EF92FF920F931F93CF93F4
:10693000DF93EC017A018B0110923A0280913A02C6
:106940008093390280913902809338028091380215
:106950008093370264E88FE00E94473461E08EE064
:106960000E946834809195048F3F19F41092A70417
:106970009AC08091950487FFF1CF81E08093A704AE
:10698000C130D10511F467E211C0C230D10551F414
:106990006FE08AE20E9447346FEB89E20E9447343D
:1069A00067E038C0C330D10531F467E08AE20E9465
:1069B00047346AEBF2CFC430D10511F463E0F6CF6F
:1069C000C530D10511F463E011C0C630D10551F4D2
:1069D00063E08AE20E94473468E989E20E94473412
:1069E00061E018C0C730D10551F460E08AE20E942E
:1069F000473468EB89E20E94473465E00BC0289772
:106A000061F460E08AE20E94473460E989E20E9412
:106A1000473462E088E20E94473460E08DE00E94E3
:106A2000473460E08CE00E944734D801C70143E05E
:106A3000B695A795979587954A95D1F78093950434
:106A40008E2D8295880F807E8093960410929704F5
:106A50001092980464E080E00E941C348FEF8093D1
:106A6000950480EE809396041092970410929804F7
:106A700064E080E20E941C3460E080E60E944734BB
:106A800061E18BE20E94473464E08FE00E9447346A
:106A900061E08EE00E9468348091950487FDF8CF14
:106AA0008BB780648BBFDF91CF911F910F91FF90C7
:106AB000EF900895AC018091A704882319F480E039
:106AC00090E008958BB78F7B8BBF209139022F5FA9
:106AD000243109F420E080913A02281711F490E063
:106AE00023C08091390290E0FC0164E0EE0FFF1FAB
:106AF0006A95E1F7E81BF90BE55CFD4FDA018FE0E1
:106B00000D9001928150E1F72093390261E080E518
:106B10000E9468348091950483FD05C040E160E1E6
:106B20008CE20E94F93391E08BB780648BBF892F90
:106B300090E008951F920F920FB60F921124EF92DA
:106B4000FF921F932F933F934F935F936F937F9386
:106B50008F939F93AF93BF93CF93DF93EF93FF9365
:106B600061E08CE20E94683480919504E82E80FFF9
:106B7000C1C0109137021F5F143109F410E08091F9
:106B80003802181709F4B1C0909137028FE0989F2E
:106B9000E0011124C959DC4F6EE080E60E946834A0
:106BA00080919704869586958695817089838981E1
:106BB000882309F45AC080919A0482958695869517
:106BC00081708A838091970490E0A0E0B0E0FBE1BF
:106BD000880F991FAA1FBB1FFA95D1F78B839C833F
:106BE000AD83BE832B813C814D815E818091980471
:106BF00090E0A0E0B0E0E3E1880F991FAA1FBB1F5F
:106C0000EA95D1F7822B932BA42BB52B8B839C83F6
:106C1000AD83BE832B813C814D815E81809199043F
:106C200090E0A0E0B0E0072E7BE0880F991FAA1F3C
:106C3000BB1F7A95D1F7702D822B932BA42BB52BEC
:106C40008B839C83AD83BE832B813C814D815E8190
:106C50008091970482958695877090E0A0E0B0E0DF
:106C6000822B932BA42BB52B0FC080919504869576
:106C70008695869581708A83809197048295869502
:106C8000877090E0A0E0B0E08B839C83AD83BE83EF
:106C90002B813C814D815E818091960490E063E080
:106CA000880F991F6A95E1F7AA2797FDA095BA2F3B
:106CB000822B932BA42BB52B8B839C83AD83BE831C
:106CC00080919A048F70888320E030E0F901E556C6
:106CD000FB4F8081F901EC0FFD1F87832F5F3F4F32
:106CE0002830310599F71093370240E061E08CE2DB
:106CF0000E94F933E4FE96C040E060E18CE20E941D
:106D0000F93390913A0280913902981709F48AC0B8
:106D100080913A029FE0899FE0011124C55CDD4F1C
:106D20008F5F80933A028B819C81AD81BE8113E09D
:106D3000B695A795979587951A95D1F78093950461
:106D40008B819C81AD81BE818295880F807E8093EE
:106D5000960489818823C9F1809196048860809384
:106D60009604209196048B819C81AD81BE81FBE1CC
:106D7000B695A79597958795FA95D1F78370822B4D
:106D800080939604209197048B819C81AD81BE8174
:106D9000E3E1B695A79597958795EA95D1F7282BC6
:106DA00020939704209198048B819C81AD81BE81B2
:106DB000072E7BE0B695A795979587957A95D1F79D
:106DC000702D282B2093980404C0109297041092E1
:106DD000980488818F70809399048A81882329F090
:106DE0008091990480648093990420E030E0F90157
:106DF000EC0FFD1F8781F901E656FB4F80832F5F63
:106E00003F4F2830310599F76DE081E50E941C3431
:106E10006BE080E50E94473480913A02843111F49E
:106E200010923A02FF91EF91DF91CF91BF91AF9114
:106E30009F918F917F916F915F914F913F912F9192
:106E40001F91FF90EF900F900FBE0F901F9018951D
:106E5000823010F482E001C08E7F82B985EC86BF5B
:106E600085B3836085BB0895DC019091A8049617D3
:106E700019F080E090E0089540E020E030E00BC0A1
:106E8000F901E555FB4F8081FD01E20FF31F80837F
:106E90004F5F2F5F3F4F491799F71092A80481E089
:106EA00090E00895DC0140E020E030E00BC0FD01FF
:106EB000E20FF31F8081F901EC54FB4F80834F5F99
:106EC0002F5F3F4F461799F76093AA0408951F92CA
:106ED0000F920FB60F9211248F939F93EF93FF930E
:106EE00081B1803629F485EC86BF1092A80453C086
:106EF00081B1803819F081B1883871F485EC86BF92
:106F00008091A804E82FF0E093B1E555FB4F908302
:106F10008F5F8093A8043FC081B1803AD1F181B1E5
:106F2000882311F485ED36C081B1883AB1F410920E
:106F3000A9049091A904E92FF0E0EC54FB4F808163
:106F400083B99F5F9093A90485EC86BF9091A904B3
:106F50008091AA049817F9F416C081B1883BC9F44E
:106F60009091A904E92FF0E0EC54FB4F808183B9A4
:106F70009F5F9093A90485EC86BF9091A9048091AE
:106F8000AA04981741F48091A90481508093A90420
:106F900002C085EC86BFFF91EF919F918F910F907A
:106FA0000FBE0F901F901895FF920F931F93982F6D
:106FB000162F042FF22E8091BD04813029F48BB757
:106FC0008F7B8BBFAF980DC0823029F48BB78F7B3E
:106FD0008BBFAE9806C0833021F48BB78F7B8BBFFD
:106FE000AD98892F0E94A810812F0E94A810802F91
:106FF0000E94A8108F2D0E94A81085B3806E85BBBB
:107000008BB780648BBF1F910F91FF900895CF9332
:10701000DF93CDB7DEB724970FB6F894DEBF0FBE6F
:10702000CDBF49835A836B837C83813011F48AE01E
:1070300005C0823011F48CE001C088E029814A81CA
:107040006B8181600E94D43724960FB6F894DEBF1E
:107050000FBECDBFDF91CF910895CF93DF93CDB712
:10706000DEB724970FB6F894DEBF0FBECDBF8823DE
:1070700011F4E0E005C0813011F4E2E001C0E4E089
:10708000842F90E09695982F882797958795A0E074
:10709000B0E09B0140E050E06CE0220F331F441F42
:1070A000551F6A95D1F7822B932BA42BB52B89837F
:1070B0009A83AB83BC8329814A816B818E2F816047
:1070C0000E94D43724960FB6F894DEBF0FBECDBF12
:1070D000DF91CF91089520E040E064E087E00E94D6
:1070E000D43720E040E060E281E10E94D43720E024
:1070F00040E060E089E00E94D43720E040E060E0BA
:107100008BE00E94D43720E040E060E08DE00E94F8
:10711000D4370895CF92DF92EF92FF920F931F938F
:10712000CF93DF936C017B018091BD04813029F402
:107130008BB78F7B8BBFAF980DC0823029F48BB794
:107140008F7B8BBFAE9806C0833021F48BB78F7BCB
:107150008BBFAD98C0E0D0E087010C0F1D1FF6017A
:10716000EC0FFD1F80810E94A810F80180832196FA
:10717000C430D10589F785B3806E85BB8BB7806439
:107180008BBFDF91CF911F910F91FF90EF90DF9018
:10719000CF900895CF93DF93CDB7DEB72C970FB67E
:1071A000F894DEBF0FBECDBF813011F48AE005C078
:1071B000823011F48CE001C088E08D83BE016F5FE6
:1071C0007F4FCE0105960E948A381C868A818B8764
:1071D0009B819A879C81998787FF03C08FEF8C875B
:1071E00001C01C8669857A858B859C852C960FB697
:1071F000F894DEBF0FBECDBFDF91CF91089580918F
:10720000C2049091C304FC0105C02C3211F4108219
:1072100004C0319620812223C1F73196F093C30434
:10722000E093C2040895CF92DF92EF92FF920F9302
:107230001F93CF93DF93CDB7DEB764970FB6F89463
:10724000DEBF0FBECDBF6B017C010E943C308823A6
:10725000E1F380E20E94ED2F2AE030E08E010F5F23
:107260001F4FA801C701B6010E94603CEE24FF2415
:1072700068010DC00E9427308823E1F70C0D1D1D09
:10728000F80180810E94ED2F0894E11CF11C0E2D65
:1072900010E0F601E00FF11F8081882359F7649612
:1072A0000FB6F894DEBF0FBECDBFDF91CF911F9117
:1072B0000F91FF90EF90DF90CF9008950F931F9361
:1072C000CF93DF93CDB7DEB724970FB6F894DEBF28
:1072D0000FBECDBF8C010E943C308823E1F3F80142
:1072E0008081805C0E94ED2FF8018181805C0E948A
:1072F000ED2FF801628170E080E090E00E94133988
:10730000F80184818C8385818B8386818A83878140
:10731000898369817A818B819C810E9413398DE0F8
:107320000E94ED2F24960FB6F894DEBF0FBECDBF9E
:10733000DF91CF911F910F910895CF92DF92EF923D
:10734000FF920F931F93CF93DF93EC0101C021961F
:107350001881812F90E00E94273D892BC1F71D32B3
:1073600029F4219681E0C82ED12C05C01B3209F4E6
:107370002196CC24DD2420E030E040E050E01AC02B
:10738000FF2400E010E080ED9FEFAFEFBFEFE80ECD
:10739000F91E0A1F1B1FCA01B9012AE030E040E0B4
:1073A00050E00E94A43C9B01AC012E0D3F1D401FEC
:1073B000511F2196E8808E2D90E0C0970A9700F328
:1073C000CD2839F050954095309521953F4F4F4F3E
:1073D0005F4FCA01B901DF91CF911F910F91FF90CB
:1073E000EF90DF90CF9008958F929F92AF92BF92CF
:1073F000CF92DF92EF92FF920F931F93CF93DF9381
:10740000CDB7DEB725970FB6F894DEBF0FBECDBF60
:107410005C01CE0101960E940930882309F4FAC06C
:107420008091BF048823A9F5098110E082E090E0F3
:107430000E94FE0F90E0805C9F4F0817190789F4A7
:107440008091C0049091C104892B09F0E3C081E0D0
:107450008093BF0480915F01882309F0DBC089819C
:10746000D7C089818D3011F08B3129F41092C1047D
:107470001092C004CFC08091C0049091C1048F3796
:10748000910508F0C7C001969093C1048093C00491
:10749000C1C080915F01882319F489810E94ED2F7A
:1074A0002981203268F08091C0049091C1048F3707
:1074B0009105A8F4FC01EC53FB4F208301960AC010
:1074C000283069F48091C0049091C104009709F4B8
:1074D00091C001979093C1048093C0048BC02D305C
:1074E00009F088C08091C0049091C104892B09F4EF
:1074F00081C080915F01813021F50E943C3088235A
:10750000E1F382E090E00E94FE0F805C0E94ED2F8C
:1075100000E010E00CC00E9427308823E1F7F8015A
:10752000EC53FB4F80810E94ED2F0F5F1F4F809126
:10753000C0049091C1040817190768F38DE00E94F8
:10754000ED2F1092C3051092C2052091C004309116
:10755000C1046091C2047091C30444EC54E090E013
:10756000A0E0B0E0240F351F2EC0913081F09130A3
:1075700018F0923031F51CC0FA018081803209F197
:10758000FD01ED5BFA4F8083119691E01AC0FA017C
:107590008081803289F4A230B10528F0FD01ED5BD5
:1075A000FA4F10821196BD016D5B7A4F92E009C0CF
:1075B000FA018081803229F0FD01ED5BFA4F808372
:1075C00011964F5F5F4F4217530779F67093C304CC
:1075D0006093C204B093C305A093C205AD5BBA4FDC
:1075E0001C9281E08093BE041092BF041092C104EB
:1075F0001092C00489818B3169F41092C1041092F9
:10760000C0041092BF0480915F01882319F48DE0BB
:107610000E94ED2F8091BE04882319F480E090E051
:10762000BCC01092BE04CC24DD2423E4822E25E0CD
:10763000922E760193E0EE0CFF1C9A95E1F7EC1880
:10764000FD08870100571E4FB801C4010E944D3C40
:10765000892B61F4F701EB56FE4F8491F701EA564E
:10766000FE4FE491982F3E2F21E00EC0F801849147
:10767000882339F00894C11CD11CFFEFCF16D10428
:10768000C1F620E090E030E0D50181E0FD011182FB
:107690008F5F11968830D1F7222309F461C0D5019C
:1076A0009C93E32E30FF40C00E94FF388C01F5010F
:1076B00080818430A1F465E872E0C8010E944D3CED
:1076C000892BB1F061E872E0C8010E944D3C892B22
:1076D000C9F06BE772E0C8010E944D3C1AC08D30C2
:1076E000F1F465E772E0C8010E944D3C892B19F462
:1076F000F501118219C060E772E0C8010E944D3C9B
:10770000892B11F481E008C069E672E0C8010E948B
:107710004D3C892B21F482E0F501818305C0C8012D
:107720000E949D39F5016183E1FE06C00E94FF3889
:107730000E949D39F5016283E2FE15C00E94FF3868
:107740000E949D396A837B838C839D838D81F501A3
:1077500083838C8184838B8185838A81868303C024
:107760008FEFD5018C938501095F1F4F82E090E078
:107770000E94FE0FF501878320E030E0F501E20F63
:10778000F31FD8018C919081890F8C932F5F3F4F0D
:107790002730310599F781E090E025960FB6F894EF
:1077A000DEBF0FBECDBFDF91CF911F910F91FF9034
:1077B000EF90DF90CF90BF90AF909F908F90089503
:1077C000A0E0B0E0E6EEFBE30C944E3DEC016881F6
:1077D00079818A819B81611571058105910549F443
:1077E00084E2A82E89EDB82E8BE5C82E87E0D82E2E
:1077F00002C05B016C01C601B5012DE133EF41E030
:1078000050E00E94EA3C27EA31E440E050E00E9468
:10781000A43C7B018C01C601B5012DE133EF41E0B1
:1078200050E00E94EA3CCA01B90124E13BE040E09B
:1078300050E00E94A43CE61AF70A080B190B17FF48
:1078400008C08FEF9FEFAFEFBFE7E80EF91E0A1FEA
:107850001B1FE882F9820A831B838FEF9FEFAFEF34
:10786000BFE7E822F9220A231B23C801B701EAE097
:10787000CDB7DEB70C946A3D0E94E03B08958CE0E2
:1078800091E00E94E03B089560930C0170930D011C
:1078900080930E0190930F010895FB01DC018D91FF
:1078A00081341CF08B350CF4805E659161341CF0E2
:1078B0006B350CF4605E861B611189F3990B08959A
:1078C000FA01CF93FF93EF93223044F1253234F540
:1078D000C22FE894CA3049F497FB3EF49095809506
:1078E000709561957F4F8F4F9F4F2C2F33274427E3
:1078F0005527FF93EF930E94053DEF91FF91605D47
:107900006A330CF0695D6193B901CA01605070403F
:107910008040904051F716F4CDE2C19310828F91D0
:107920009F91CF910C94943CDC01FC01672F7191E5
:107930007723E1F7329704C07C916D937083629155
:10794000AE17BF07C8F30895629FD001739FF0017F
:10795000829FE00DF11D649FE00DF11D929FF00DDF
:10796000839FF00D749FF00D659FF00D9927729F16
:10797000B00DE11DF91F639FB00DE11DF91FBD01A1
:10798000CF0111240895AA1BBB1B51E107C0AA1FF8
:10799000BB1FA617B70710F0A61BB70B881F991FB0
:1079A0005A95A9F780959095BC01CD01089597FB54
:1079B000092E07260AD077FD04D0E5DF06D0002087
:1079C0001AF4709561957F4F0895F6F7909581951B
:1079D0009F4F089597FB092E05260ED057FD04D022
:1079E00014D00AD0001C38F450954095309521955C
:1079F0003F4F4F4F5F4F0895F6F7909580957095E4
:107A000061957F4F8F4F9F4F0895A1E21A2EAA1BB9
:107A1000BB1BFD010DC0AA1FBB1FEE1FFF1FA2173E
:107A2000B307E407F50720F0A21BB30BE40BF50B3B
:107A3000661F771F881F991F1A9469F760957095C4
:107A4000809590959B01AC01BD01CF0108959111E6
:107A50001AC0803219F089508550D0F70895E19905
:107A6000FECFBFBBAEBBE09A11960DB20895E1996F
:107A7000FECFBFBBAEBB0DBA11960FB6F894E29A1B
:107A8000E19A0FBE08959927882708952F923F9273
:107A90004F925F926F927F928F929F92AF92BF921E
:107AA000CF92DF92EF92FF920F931F93CF93DF93CA
:107AB000CDB7DEB7CA1BDB0B0FB6F894DEBF0FBE27
:107AC000CDBF09942A88398848885F846E847D8474
:107AD0008C849B84AA84B984C884DF80EE80FD8076
:107AE0000C811B81AA81B981CE0FD11D0FB6F894EC
:0C7AF000DEBF0FBECDBFED010895FFCF3B
:107AFC00C1116C2522253A1BF32D8A26C2220122A4
:107B0C003821331F801D5B1C441BF01AFD28812873
:107B1C00C311C511C711C911EE133514BA14C3140E
:107B2C00DF14F214F914C419001500199D1841182A
:107B3C000226C6126228192103153E154B154C1549
:107B4C004E15501552155415561558155A155C15D9
:107B5C005E15601562156415661568156A156C1549
:107B6C006E15701572157415761578157A157C15B9
:107B7C002C0433042D042E042F043004310432045D
:107B8C007E15811591159515CB17BA15A017C11532
:107B9C0077178D1811162716DD1635160100000003
:00000001FF
